:100000000C94E1000C9409010C9409010C94090171
:100010000C9409010C9409010C9409010C94090138
:100020000C9409010C9409010C9409010C94090128
:100030000C9409010C9409010C9409010C94090118
:100040000C940B260C9409010C94F7280C94292984
:100050000C9409010C9409010C9409010C940901F8
:100060000C946C1E0C940901D5060A070A070A07AE
:100070000A070A070A077E060A07AB060A070A07E5
:1000800005060A0791060A070A070A070A070A0768
:100090000A070A070A070A070A070A070A07F205F2
:1000A0000A074F06D8050A07CA060A07E9050A071C
:1000B0000A070A070A0779060A07AB0683060A0732
:1000C00005069A0688060A070A070A070C07E806C3
:1000D000F90604200A20102016201C2022202920A6
:1000E00007634236B79BD8A71A39685618AEBAAB21
:1000F000558C1D3CB7CC5763BD6DEDFD753EF617B5
:100100007231BF000000803F08000000BE92244909
:10011000123EABAAAA2ABECDCCCC4C3E0000008039
:10012000BEABAAAAAA3E00000000BF000000803FAC
:100130000000000000084178D3BB4387D1133D196C
:100140000E3CC3BD4282AD2B3E68EC8276BED98F99
:10015000E1A93E4C80EFFFBE01C4FF7F3F000000DD
:100160000000000000080002010000030407000076
:10017000000000000000010204081020408001027D
:1001800004081020010204081020040404040404DC
:100190000404020202020202030303030303000039
:1001A0000000230026002900000000002500280090
:1001B0002B0000000000240027002A0053058A1DA0
:1001C000592911241FBECFEFD8E0DEBFCDBF14E008
:1001D000A0E0B1E0E4EFFCE602C005900D92AE3184
:1001E000B107D9F726E0AEE1B4E001C01D92A13914
:1001F000B207E1F711E0C2ECD1E004C02297FE01A2
:100200000E944031CC3BD107C9F70E949D290C9434
:1002100078360C940000CF93C82F809320050E945D
:100220000A1B8C2F0E940A1B6C2F88E994E00E9405
:10023000071A6C2F82E494E0CF910C94071AEF9286
:10024000FF920F931F93CF93DF9300D000D0CDB7D1
:10025000DEB7182F7901013069F488E994E0498309
:100260005A836B837C830E94701849815A8101975D
:10027000E1F509C00230C9F588E994E00E947018E0
:10028000029799F517C0113021F4BA0188E994E07A
:1002900005C0123051F5BA0182E494E00F900F903E
:1002A0000F900F90DF91CF911F910F91FF90EF90E2
:1002B0000C945816113031F4F7014181608188E9BE
:1002C00094E007C0123089F4F7014181608182E433
:1002D00094E00F900F900F900F90DF91CF911F91AE
:1002E0000F91FF90EF900C944E180F900F900F907D
:1002F0000F90DF91CF911F910F91FF90EF90089594
:10030000FF920F931F93CF93DF93CDB7DEB7C458FF
:10031000D1090FB6F894DEBF0FBECDBFF82E092F5E
:10032000162F60E088E994E00E941818EF2DF02F56
:10033000819189836FEF610FCC57DF4F6883C45879
:10034000D040DE01149680E090E070E086179707B9
:1003500024F421912D930196F9CF2091140130912D
:100360001501409116015091170168E974E0CE0122
:1003700001960E949B0B61E088E994E00E941818A6
:10038000CC57DF4F0FB6F894DEBF0FBECDBFDF9165
:10039000CF911F910F91FF900895CF93DF9300D0DD
:1003A00000D000D0CDB7DEB768E171E080EF95E016
:1003B0000E94F8296BE171E080EF95E00E94F82936
:1003C0006EE280EF95E00E94FA2960E371E080EF31
:1003D00095E00E94F82968E471E080EF95E00E94C2
:1003E000F82968E974E0CE0101960E947418BE01F4
:1003F0006F5F7F4F80EF95E00E94EA29CE01019662
:100400000E940F2C66E371E080EF95E00E94F829CE
:1004100088E994E00E94101AAB01BC012AE030E0A8
:1004200080EF95E00E94F62A80911B0590911C05B3
:10043000892BF9F06AE371E080EF95E00E94F829DA
:1004400060911B0570911C054AE050E080EF95E03B
:100450000E940A2B6EE371E080EF95E00E94F8297C
:100460004AE050E060910F0180EF95E00E94032B7D
:1004700012C060E471E080EF95E00E94F82988E9FD
:1004800094E00E940A1AAB01BC012AE030E080EF40
:1004900095E00E94F62A64E471E080EF95E00E9406
:1004A000F82982E494E00E947119882309F466C057
:1004B00066E471E080EF95E00E94F82962E474E060
:1004C000CE0101960E947418BE016F5F7F4F80EFCE
:1004D00095E00E94EA29CE0101960E940F2C66E366
:1004E00071E080EF95E00E94F82982E494E00E9498
:1004F000101AAB01BC012AE030E080EF95E00E94C9
:10050000F62A8091190590911A05892BF9F06AE372
:1005100071E080EF95E00E94F829609119057091D3
:100520001A054AE050E080EF95E00E940A2B6EE346
:1005300071E080EF95E00E94F8294AE050E0609178
:100540000E0180EF95E00E94032B12C060E471E081
:1005500080EF95E00E94F82982E494E00E940A1A54
:10056000AB01BC012AE030E080EF95E00E94F62A62
:1005700064E471E080EF95E00E94F82982E294E063
:100580000E94190E882331F06BE471E080EF95E052
:100590000E94F8296DE580EF95E00E94392A2696A1
:1005A0000FB6F894DEBF0FBECDBFDF91CF91089597
:1005B000CF92DF92EF92FF920F931F93CF93DF932F
:1005C000CDB7DEB7C154D1090FB6F894DEBF0FBE68
:1005D000CDBF8C0160E00E941818BE016F5F7F4F95
:1005E000C8010E94251580911705882329F0CE01A6
:1005F00001960E941211A7C080911D0561E0813013
:1006000011F581E494E00E948A0FCE0101967C01ED
:100610006E0191E4C90ED11CF70161917F0140E1A7
:1006200050E080EF95E00E94032B60E673E080EFDE
:1006300095E00E94F829EC14FD0471F780EF95E035
:100640000E94012A80C081E494E00E948A0F809178
:100650002005882319F165E571E080EF95E00E949F
:10066000F829CE0101967C016E0191E1C90ED11CE1
:10067000F70161917F0140E150E080EF95E00E9439
:10068000032B60E673E080EF95E00E94F829EC14FC
:10069000FD0471F780EF95E00E94012AC8010E94D5
:1006A0000A1A0E948B12882341F0CE0101960E9403
:1006B0005E12882311F045E024C0C8010E940A1A86
:1006C0000E943922811153C0C8010E940A1A0E9457
:1006D0006623882331F0CE0101960E9439238111CF
:1006E0008BC0C8010E940A1A0E940E15882309F4C3
:1006F0004AC0CE0101960E94E114882309F443C048
:1007000046E0809118058823F1F04423E1F060E48D
:1007100070E080E090E022964FAF22970E948426FE
:1007200022964FAD2297BE016F5F7F4FC8010E9496
:100730002B1A80912005882331F064E771E080EF67
:1007400095E00E94272A61E0C8010E941818CF5B3B
:10075000DF4F0FB6F894DEBF0FBECDBFDF91CF9154
:100760001F910F91FF90EF90DF90CF900895CE01F1
:1007700001960E940C22882309F4A6CFCE0101968F
:100780000E94991F3FC0C8010E940A1A0E94EB0DE7
:10079000882331F0CE0101960E94BE0D81112EC03A
:1007A000C8010E940A1A0E948B12882331F0CE01E0
:1007B00001960E94DE258111A3CFC8010E940A1A6A
:1007C0000E94AE1C882331F0CE0101960E94811C4C
:1007D000811116C0C8010E940A1A0E94090C8823C0
:1007E00099F0CE0101960E94390B882369F0CE0161
:1007F00001960E94AF0A06C04AE083CF4CE081CF49
:1008000044E07FCF482F7DCF80911D05823011F0CD
:1008100040E077CFCE0101967C016E0191E4C90ED4
:10082000D11CF70161917F0140E150E080EF95E03C
:100830000E94032B60E673E080EF95E00E94F829A8
:10084000EC14FD0471F780EF95E00E94012AE0CFDF
:100850004F925F926F927F928F929F92AF92BF92D0
:10086000CF92DF92EF92FF920F93CF93DF934C01E1
:100870005B01EA0179012115310509F470C00E947C
:100880005526F5014080518062807380641575059E
:100890008605970520F410821182128213820E942D
:1008A000552648EE53E0E49E9001E59E300DF49EFF
:1008B000300D1124F501C080D180E280F380C20E9A
:1008C000D31EE11CF11CC616D706E806F90608F08F
:1008D00046C0C880D980EA80FB80FAE8CF16F2E2F1
:1008E000DF06E104F10491F401FF05C08BE695E217
:1008F000A0E0B0E006C000FF24C089E593E4A0E0DA
:10090000B0E088839983AA83BB831BC08BE6C8169B
:1009100085E2D806E104F10449F400FDEECF02FFC0
:1009200010C08AE892E2A0E0B0E0EBCFE9E5CE1695
:10093000E3E4DE06E104F10421F402FDF2CF01FD5F
:10094000D5CF488159816A817B81C4010E941717E4
:100950000E945526F5016083718382839383DF9122
:10096000CF910F91FF90EF90DF90CF90BF90AF901D
:100970009F908F907F906F905F904F90089526E0AA
:1009800040E051EE60E070E080EF95E00E94952835
:1009900068EC70E080E090E00E9484268091200561
:1009A000882331F06CE771E080EF95E00E94272A00
:1009B000809120050E940B011092250582E294E0AF
:1009C0000E94020E60911E0570911F0582E294E064
:1009D0000E941C0E61E081E494E00E94BA0F0E9424
:1009E0005526609313057093140580931505909315
:1009F000160588E994E00E948E18409110015091EC
:100A00001101609112017091130188E994E00E9434
:100A1000761740910A0150910B0160910C01709181
:100A20000D0188E994E00E94171761E088E994E0DD
:100A30000E94181882E494E00E947119882309F139
:100A400082E494E00E948E184091100150911101AF
:100A5000609112017091130182E494E00E94761774
:100A600040910601509107016091080170910901C0
:100A700082E494E00E94171761E082E494E00E940F
:100A8000181880912005882331F06FEB71E080EF1A
:100A900095E00E94272A68EE73E080E090E00E94D3
:100AA00084260C94CD01CF92EF920F93CC24C39463
:100AB00082E0E82E0AE02DE04CE06BE088E994E06B
:100AC0000E947919C12C93E0E92E08E02DE04CE05A
:100AD0006BE082E494E00E94791981E494E00E9442
:100AE000740F82E294E00F91EF90CF900C94F40D8C
:100AF0000F931F93CF93DF9300D000D0CDB7DEB715
:100B000080EF95E00E94B227892B09F493C180EF12
:100B100095E00E94CB27082F8C3269F4E091EE0417
:100B200081E08E0F8093EE04F0E0E151FB4F809165
:100B30001E04808371C180ED800F8A3010F52091F2
:100B40001E0430911F044091200450912104AAE01A
:100B5000B0E00E9444316053710981099109112765
:100B600007FD1095212F312F600F711F821F931FDA
:100B700060931E0470931F048093200490932104BB
:100B800059C1802F8F7D81548A3108F04EC1402F8A
:100B9000552747FD5095652F752FFA01E654F10949
:100BA000E533F10508F036C1EC5CFF4F0C943E31A3
:100BB00081E040911E0450911F04609120047091C7
:100BC0002104452B462B472B09F480E00E940B01A2
:100BD00023C160911E0470911F0482E294E00E9480
:100BE0001C0E1AC161E080911E0490911F04A09117
:100BF0002004B0912104892B8A2B8B2B09F460E00F
:100C000081E494E00E94BA0F07C140911E04509104
:100C10001F04609120047091210441305105610549
:100C2000710581F050F0423051056105710571F494
:100C30004AE852E260E070E009C049E553E460E050
:100C400070E004C04BE655E260E070E0023759F412
:100C500040930A0150930B0160930C0170930D01B6
:100C600088E994E019C082E494E049835A836B8355
:100C70007C830E94711949815A816B817C81882310
:100C800009F4CAC04093060150930701609308011C
:100C90007093090182E494E00E941717BDC080910F
:100CA0001E0490911F04A0912004B0912104813072
:100CB0009105A105B10581F050F082309105A105A3
:100CC000B10571F48AE892E2A0E0B0E009C089E5DC
:100CD00093E4A0E0B0E004C08BE695E2A0E0B0E0D1
:100CE0008093140190931501A0931601B0931701FE
:100CF00093C080911E0480930F018EC080911E04CA
:100D000080930E0189C080911E0480931D0584C0CC
:100D100080911E0490911F0490931C0580931B05E5
:100D20007BC080911E0490911F0490931A058093BC
:100D3000190572C06091EE04E62FF0E0E151FB4F1F
:100D400080911E0480836F5F6093EE048FEE94E0C9
:100D50000E9480011CC09091EE0440911E045091AD
:100D60001F046091200470912104E92FF0E0E1510B
:100D7000FB4F40839F5F9093EE040F3411F482E0A9
:100D800001C081E0092F2FEE34E00E941F01109274
:100D9000EE0442C040911E0450911F046091200453
:100DA0007091210488E994E010C082E494E00E94EC
:100DB0007119882389F140911E0450911F0460919C
:100DC00020047091210482E494E00E94761724C0EC
:100DD00021E080911E0490911F04A0912004B09105
:100DE0002104892B8A2B8B2B09F420E020931805F2
:100DF00013C021E080911E0490911F04A091200453
:100E0000B0912104892B8A2B8B2B09F420E02093AD
:100E1000170502C00E94CD0110921E0410921F04FB
:100E2000109220041092210405C00152003210F4E7
:100E30000E94CD0182E294E00E94470F88E994E08D
:100E40000E94961688E994E00E943715882321F0C5
:100E500088E994E00E94D80282E494E00E9471192B
:100E6000882371F082E494E00E94961682E494E074
:100E70000E943715882321F082E494E00E94D80272
:100E800020911B0530911C0500910F014AE051E0B3
:100E900063E175E088E994E00E9428042091190537
:100EA00030911A0500910E0146E051E06FE075E0C7
:100EB00082E494E00E9428040F900F900F900F900E
:100EC000DF91CF911F910F910895FC011082118243
:100ED000128213820895FC014083518362837383DD
:100EE0000895CF92DF92EF92FF92FC01808D918D59
:100EF000481B590B61097109A689B7899A01AB0191
:100F00000E9444316B017C018FE0F594E794D79403
:100F1000C7948A95D1F760897189882777FD809574
:100F2000982F2BE0660F771F881F991F2A95D1F7FE
:100F300022893389442737FD4095542F2C0D3D1DC0
:100F40004E1D5F1D0E941F312C0D3D1D4E1D5F1D4E
:100F5000CA01B901FF90EF90DF90CF9008951F93E1
:100F6000CF93DF931F92CDB7DEB7162F67E770E000
:100F700087E295E049830E94721D612F87E295E028
:100F80000E940F1D4981642F87E295E00E940F1D8A
:100F900087E295E00F90DF91CF911F910C94871D10
:100FA000CF93C62F67E770E087E295E00E94721D3D
:100FB0006C2F87E295E00E940F1D87E295E00E946A
:100FC000871D67E770E087E295E00E94721D41E0AF
:100FD00050E067E770E087E295E00E94651D87E2D8
:100FE00095E00E94BF1CC82F87E295E00E94871DF4
:100FF0008C2FCF910895CF93DF93C62F67E770E0D2
:1010000087E295E00E94721D6C2F87E295E00E94B6
:101010000F1D87E295E00E94871D67E770E087E279
:1010200095E00E94721D42E050E067E770E087E2C1
:1010300095E00E94651D87E295E00E94BF1CD82FB5
:1010400080E0C82F87E295E00E94BF1CC82BD92BF7
:1010500087E295E00E94871DCE01DF91CF91089530
:10106000CF93DF93EC0187E295E00E944E1D60ED87
:10107000CE010E94D007853509F044C06AEACE014E
:101080000E94FB079D838C836CEACE010E94FB07C4
:101090009F838E836EEACE010E94FB079987888723
:1010A00060EBCE010E94FB079D8B8C8B62EBCE0127
:1010B0000E94FB079F8B8E8B64EBCE010E94FB0787
:1010C000998F888F66EBCE010E94FB079B878A87EA
:1010D00068EBCE010E94FB079D878C876AEBCE01EF
:1010E0000E94FB079F878E876CEBCE010E94FB0757
:1010F000998B888B6EEBCE010E94FB079B8B8A8BB2
:1011000081E001C080E0DF91CF910895CF93DF931C
:10111000EC014EE264EF0E94AF0765E070E080E012
:1011200090E00E94842666EFCE01DF91CF910C946F
:10113000FB07CF93DF93EC010E948608AC0160E0CF
:1011400070E0CE010E947107685F7F4F8F4F9F4F05
:1011500034E095958795779567953A95D1F70E94F4
:101160006D2E20E030E040E251E40E94D22DDF916C
:10117000CF910895CF92DF92EF92FF92CF93DF93BA
:10118000EC0144EB64EF0E94AF076EE070E080E09A
:1011900090E00E94842666EFCE010E94FB076C015E
:1011A000E12CF12CFE2CED2CDC2CCC2468EFCE01B4
:1011B0000E94D007A7019601282BCA01B90156E069
:1011C00096958795779567955A95D1F7DF91CF9149
:1011D000FF90EF90DF90CF9008952F923F924F9223
:1011E0005F926F927F928F929F92AF92BF92CF92B7
:1011F000DF92EF92FF920F931F93CF93DF93CDB7C0
:10120000DEB72C970FB6F894DEBF0FBECDBF1C0122
:101210000E9486088C01C1010E94BA086D837E83FA
:101220008F839887A80160E070E0C1010E94710778
:101230004B015C0180EA881A8FE0980AA108B10886
:10124000A5019401C501B4010E94ED302B013C01C0
:101250000CE075946794579447940A95D1F7D1019F
:1012600014960D911C91159718960D90BC91A02D78
:101270000E944F316B017C018DE0F594E794D79487
:10128000C7948A95D1F7F101A285B385A301920194
:101290000E944F31BB2797FDB095AB2FC80ED91ECA
:1012A000EA1EFB1EF2E0CF0ED11CE11CF11C32E065
:1012B000F594E794D794C7943A95D1F780E8D80E7F
:1012C000E11CF11CF101A489B589A70196010E94D6
:1012D0004431DC01CB014FE0B695A79597958795F2
:1012E0004A95D1F789839A83AB83BC836801EE2446
:1012F000D7FCE094FE2C52E0CC0CDD1CEE1CFF1C55
:101300005A95D1F7A485B585A30192010E944F316A
:101310002B013C016BE075946794579447946A9550
:10132000D1F7A681B781A50194010E944F31EBE06E
:101330009595879577956795EA95D1F7460E571E4F
:10134000681E791EC40CD51CE61CF71CF2E0CC0C00
:10135000DD1CEE1CFF1CFA95D1F792E0C90ED11CE2
:10136000E11CF11CC701B60124E030E040E050E090
:101370000E941F318D819E81AF81B885821B930BA6
:10138000A40BB50B9C01AD01A4EDB0E30E94443168
:1013900097FD0DC0660F771F881F991F29813A811D
:1013A0004B815C810E94FD3049015A010CC02981AA
:1013B0003A814B815C810E94FD3049015A01880CC1
:1013C000991CAA1CBB1C9927B7FC9A958B2D7A2DCA
:1013D000692D9B01AC010E94ED309B01AC01AEED8B
:1013E000BBE00E9444316C01FF24D7FCF094EF2C49
:1013F000A3E4B3EEA50194010E945231BB2797FDEF
:10140000B095AB2FC80ED91EEA1EFB1E9FECC90E6D
:101410009EE0D91EE11CF11CA4E0F594E794D7945A
:10142000C794AA95D1F7D1016D917D918D919C9131
:101430000E946D2E20E03AE24DE257E40E94D22D48
:101440009B01AC0160E070E080E89FE30E94692DA1
:1014500026EF38E248EA50E40E94842F9B01AC0159
:10146000C501B4016C0D7D1D8E1D9F1D29873A8716
:101470004B875C870E946D2E29853A854B855C855C
:101480000E94D22D0E943A2E0E946D2E20E030E064
:1014900048EC52E40E94D22D0E943A2E2C960FB6B0
:1014A000F894DEBF0FBECDBFDF91CF911F910F919A
:1014B000FF90EF90DF90CF90BF90AF909F908F9074
:1014C0007F906F905F904F903F902F900895DF92A4
:1014D000EF92FF920F931F93CF93DF938C01EB0159
:1014E00081E08A8318821982F801628184E0860F84
:1014F000E82EF12CEE0DFF1D3197D080D9826D5F63
:10150000C8010E94F11AD8121A82F80180818C3C1D
:1015100009F01A828A818823D1F0F80181818883B9
:101520008281FE01ED57FF4F808383E090E0F1E080
:10153000EF1AF1088E159F0554F4F801E80FF91F12
:101540002081FE01E80FF91F20830196F3CFDF9180
:10155000CF911F910F91FF90EF90DF900895FC01C4
:1015600082818C5F0895CF92DF92EF92FF920F936A
:101570001F93CF93DF93EC017B0161E673E00E9440
:101580007D2C62EF71E0CE010E94E62CF7016081B4
:10159000CE010E94092D60E673E0CE010E94E62C88
:1015A00000E010E06701F3E8CF0ED11CF601808166
:1015B00090E0081719077CF4F701E00FF11F638131
:1015C000CE010E94092D60E673E0CE010E94E62C58
:1015D0000F5F1F4FEBCFCE01DF91CF911F910F9186
:1015E000FF90EF90DF90CF900895EF92FF920F93CE
:1015F0001F93CF93DF93CDB7DEB7CA58D1090FB68B
:10160000F894DEBF0FBECDBF8C017B0161E673E0B5
:101610000E947D2CF70180818C3CE1F4BE016F5F5C
:101620007F4FC7010E94670A8B81882399F0BE0112
:101630006F5F7F4FCE018B579F4F0E94B30ABE0151
:101640006B577F4FC8010E94932CCE018B579F4F41
:101650000E940F2CC801C657DF4F0FB6F894DEBFAB
:101660000FBECDBFDF91CF911F910F91FF90EF90F3
:1016700008951F93CF93DF9300D000D000D0CDB753
:10168000DEB7BC01CE0101960E94F50A8D819E81D4
:10169000892B39F0BE016F5F7F4F80EF95E00E948C
:1016A000152A11E02D813E81232B09F410E0CE0193
:1016B00001960E940F2C812F26960FB6F894DEBF5C
:1016C0000FBECDBFDF91CF911F910895CF93DF93D0
:1016D000FB01DB0120E030E01D922F5F3F4F2038FF
:1016E0003105D1F72CEC2083DC012C912183AD57FF
:1016F000BF4F2C912283AF014D5F5F4F20E030E060
:101700006C91C62FD0E02C173D0754F4EC01C20FAA
:10171000D31F6B81EA016993AE012F5F3F4FF0CF7A
:101720002396CE0FDF1F6D5FCF010E94F11A8883D1
:10173000DF91CF910895CF92DF92EF92FF920F93B6
:101740001F93CF93DF93CDB7DEB7C458D1090FB63F
:10175000F894DEBF0FBECDBF8B01BE016F5F7F4F20
:10176000CF57DF4F2883C158D040CE57DF4F388343
:10177000C258D040CD57DF4F4883C358D040CC57D4
:10178000DF4F5883C458D0400E94660B60E0C80108
:101790000E941818C8010E940A1A6B017C01CF57D9
:1017A000DF4F2881C158D040CE57DF4F3881C25813
:1017B000D040CD57DF4F4881C358D040CC57DF4F82
:1017C0005881C458D040BA01A901C8010E94171716
:1017D0004B814C5FBE016F5F7F4FC8010E942B1A87
:1017E000B701A601C8010E94171761E0C8010E9455
:1017F0001818CC57DF4F0FB6F894DEBF0FBECDBF21
:10180000DF91CF911F910F91FF90EF90DF90CF90DC
:10181000089581E0089520E030E040E0FC0151911E
:10182000CF01450F2F5F3F4F2C303105B9F781E0D5
:10183000411180E008950F931F93CF93DF938C01A4
:10184000EB0181E0898FF801808188838181898320
:101850008481282F221F2227221F2D83828190E03E
:10186000982F88273381832B9B838A83918581E0FE
:1018700096FF80E08E8BF8019185892F881F88273D
:10188000881F8F8B2223A1F01E821F821886198643
:101890001A861B861C861D861E861F86188A198A34
:1018A0001A8A1B8A1C8A1D8A1C82188E198E61C096
:1018B000F801608570E080E090E00E946D2E20E0ED
:1018C00030E040E05FE30E94212F20E030E040E084
:1018D00053E40E946A2D6E837F8388879987F8017D
:1018E000668170E0762F66278781682B882777FDD1
:1018F0008095982F0E946D2E6A877B878C879D87A5
:10190000F80164816F7370E0762F66278581682BFC
:1019100075956795882777FD8095982F0E946D2E85
:101920006E877F87888B998BF80161856F7370E074
:10193000762F66278285682B882777FD8095982FDC
:101940000E946D2E20E030E048EC52E40E94D22D3F
:101950006A8B7B8B8C8B9D8BF801948181E096FF49
:1019600080E08C83F8018385888FC8010E940B0C6E
:10197000898FF80186818A3A21F487818A3A09F4AD
:10198000198EDF91CF911F910F910895FF920F93C0
:101990001F93CF93DF93EC018B0161E673E00E940C
:1019A0007D2C67E872E0CE010E94E62CF80163818D
:1019B000CE010E94092D60E673E0CE010E94E62C64
:1019C000F8016281CE010E94092D60E673E0CE012C
:1019D0000E94E62C20E030E040E251E4F80166810C
:1019E0007781808591850E94212F0E943A2EF62EC4
:1019F000672FCE010E94092D60E673E0CE010E94A0
:101A0000E62C6F2DCE010E94092D60E673E0CE0119
:101A10000E94E62CF80162857385848595850E9475
:101A20003A2E672FCE010E94092D60E673E0CE01A9
:101A30000E94E62CF80162857385848595850E9455
:101A40003F2ECE010E94092D60E673E0CE010E9478
:101A5000E62CF80166857785808991890E943A2E67
:101A6000672FCE010E94092D60E673E0CE010E942F
:101A7000E62CF80166857785808991890E943F2E42
:101A8000CE010E94092D60E673E0CE010E94E62C93
:101A900020E030E048EC52E4F801628973898489DF
:101AA00095890E94212F0E943A2EF62E672FCE0193
:101AB0000E94092D60E673E0CE010E94E62C6F2D96
:101AC000CE010E94092D60E673E0CE010E94E62C53
:101AD000F8016581660F8481680FCE010E94092D8F
:101AE000CE01DF91CF911F910F91FF900895EF925A
:101AF000FF920F931F93CF93DF93CDB7DEB7A097DD
:101B00000FB6F894DEBF0FBECDBF8C017B0161E63E
:101B100073E00E947D2CF7018081853209F5818177
:101B2000982F9F7B9A3211F08034D1F4BE016F5F01
:101B30007F4FC7010E941B0C8A8D882389F0BE014C
:101B40006F5F7F4FCE014B960E94C60CBE01655E53
:101B50007F4FC8010E94932CCE014B960E940F2C00
:101B6000C801A0960FB6F894DEBF0FBECDBFDF91BF
:101B7000CF911F910F91FF90EF9008951F93CF93F6
:101B8000DF9300D000D000D0CDB7DEB7BC01CE01CE
:101B900001960E94770D8D819E81892B39F0BE01BF
:101BA0006F5F7F4F80EF95E00E94152A11E02D8135
:101BB0003E81232B09F410E0CE0101960E940F2CE8
:101BC000812F26960FB6F894DEBF0FBECDBFDF91F2
:101BD000CF911F91089521E06B36754281059105E3
:101BE00009F020E0822F0895CF93DF93EC01019656
:101BF0000E94650718821B8E1C8E1D8E1E8EDF9123
:101C0000CF9108950F931F93CF93DF93EC018C0135
:101C10000F5F1F4F40E050E0BA01C8010E946B0700
:101C2000C8010E9430088883DF91CF911F910F91E6
:101C30000895FC0180810895AB01662757FD6095EA
:101C4000762F01960C946B07AF92BF92CF92DF92E2
:101C5000EF92FF920F931F93CF93DF931F92CDB715
:101C6000DEB75C018A0161E673E00E947D2CF80119
:101C7000C680D780E084F18420E030E040E252EC7E
:101C8000C701B6010E94CE2D87FD7EC020E030E066
:101C90004AEA52E4C701B6010E941D2F18160CF43F
:101CA00073C063E972E0C5010E94E62CF80160810F
:101CB000C5010E94092D6AE972E0C5010E94E62C67
:101CC00020E030E040E251E4F801668177818085D0
:101CD00091850E94212F20E030E04AE754E40E94E1
:101CE0006A2D0E943A2EF62EE72E60E673E0C501BB
:101CF0000E94E62C6E2DC5010E94092D60E673E05E
:101D0000C5010E94E62C6F2DC5010E94092D61EAD4
:101D100072E0C5010E94E62C6DE972E0C5010E94E7
:101D2000E62C6DE972E0C5010E94E62C6DE972E0D7
:101D3000C5010E94E62C6DE972E0C5010E94E62C07
:101D4000F8012181828181112C5F60E673E0C50179
:101D500029830E94E62C2981622FC5010E94092D4A
:101D600060E673E0C5010E94E62CF8016385C501B9
:101D70000E94092D60E673E0C5010E94E62CF8017F
:101D80006285C5010E94092DC5010F90DF91CF9199
:101D90001F910F91FF90EF90DF90CF90BF90AF9089
:101DA00008958F929F92AF92BF92CF92DF92EF925F
:101DB000FF920F931F93CF93DF93CDB7DEB7629758
:101DC0000FB6F894DEBF0FBECDBF7C018B0161E67C
:101DD00073E00E947D2CF8018081882309F443C0C0
:101DE0000E945526F801838C948CA58CB68CF0E16A
:101DF0008F0EF7E29F1EA11CB11C681579058A059C
:101E00009B0588F10E945526F801638F748F858F9A
:101E1000968F19821B821A8281E08C836801FFEF02
:101E2000CF1ADF0AC6010E9499086F8378878987D5
:101E30009A87C6010E94ED087C876B878C81882376
:101E400091F0AE014F5F5F4FB801CE010D960E9439
:101E5000240EBE01635F7F4FC7010E94932CCE0109
:101E60000D960E940F2CC70162960FB6F894DEBF44
:101E70000FBECDBFDF91CF911F910F91FF90EF90DB
:101E8000DF90CF90BF90AF909F908F9008951F9359
:101E9000CF93DF9300D000D000D0CDB7DEB7BC0128
:101EA000CE0101960E94D10E8D819E81892B39F041
:101EB000BE016F5F7F4F80EF95E00E94152A11E011
:101EC0002D813E81232B09F410E0CE0101960E9462
:101ED0000F2C812F26960FB6F894DEBF0FBECDBF14
:101EE000DF91CF911F91089521E0FC012083089597
:101EF000CF93C62FFC018081882351F061E089E0F7
:101F00000E941A2761E06C2789E0CF910C94532737
:101F1000CF910895EF92FF920F931F93CF93DF938A
:101F20008C01662301F16B3008F06AE0C0E0D0E07C
:101F3000E62EF12CCE15DF05B4F461E0C8010E9455
:101F4000780F62E370E080E090E00E94842660E019
:101F5000C8010E94780F62E370E080E090E00E9488
:101F600084262196E7CFDF91CF911F910F91FF90AB
:101F7000EF900895FC016083611102C00C94780F0A
:101F8000089564E00C94F11ABF92CF92DF92EF9221
:101F9000FF920F931F93CF93DF938C01EB0181E0AE
:101FA0008B87F801F480FA86C8010E94C10FF812ED
:101FB0001B861982F80180818F70F4E08F9FC00129
:101FC0001124898330912505F8012181922F332333
:101FD00011F0907C04C09295969596959370982BED
:101FE0009983F801808182958F708883893009F008
:101FF0001B86F801818185FB882780F98A8381818E
:10200000829581708B83B28061816F7070E080E017
:1020100090E00E946D2E20E030E048EC52E40E94F7
:10202000212F20E030E0A9010E946A2D6B017C0184
:102030006B2D62956F7070E080E090E00E946D2ED5
:1020400020E030E040E251E40E94212F9B01AC01EE
:10205000C701B6010E946A2D6B017C016B2D6F7068
:1020600070E080E090E00E946D2E9B01AC01C70102
:10207000B6010E946A2D20E030E040E251E40E9467
:10208000D22D20E030E040E252E40E94692D6C83C2
:102090007D838E839F83F8019381892F881F8827F2
:1020A000881F888783818F778987DF91CF911F91E0
:1020B0000F91FF90EF90DF90CF90BF900895AF9277
:1020C000BF92CF92DF92EF92FF920F931F93CF9325
:1020D000DF9300D000D000D0CDB7DEB75C018B011C
:1020E00061E673E0CE0101960E947D2C66EA72E003
:1020F000CE0101960E94E62CF8016181CE01019685
:102100000E94092D60E2CE0101960E94F62CF80192
:1021100081858F77843610F08A3651F4F8018281F8
:10212000882319F061E870E008C061E070E005C044
:102130008D3709F042C062E870E0CE0101960E943E
:10214000362D60E2CE0101960E94F62C20E030E0B0
:1021500040E251E4F80164817581868197810E9493
:10216000212F20E030E04AE754E40E946A2D0E94CB
:102170003F2EF62E672FCE0101960E94092D60E2B8
:10218000CE0101960E94F62C6F2DCE0101960E9481
:10219000092D60E2CE0101960E94F62CF801C48060
:1021A000D580E680F78020E030E040E752E4C701C8
:1021B000B6010E941D2F87FD06C061E673E0C501D0
:1021C0000E947D2C19C020E030E040E252ECC701B3
:1021D000B6010E94CE2D181684F7F801618580851E
:1021E00081116068CE0101960E94092DBE016F5FCA
:1021F0007F4FC5010E94AA2CCE0101960E940F2C90
:10220000C50126960FB6F894DEBF0FBECDBFDF9195
:10221000CF911F910F91FF90EF90DF90CF90BF90E3
:10222000AF900895EF92FF920F931F93CF93DF9398
:10223000CDB7DEB7A1970FB6F894DEBF0FBECDBF06
:102240007C01BE016F5E7F4F0E94C40F1D8E1E8EEB
:102250001F8E18A219A22A89FE017D96CE018296B0
:102260003191231709F4DBC0E817F907C9F70E9479
:1022700055260091210510912205209123053091CA
:102280002405601B710B820B930B9F938F937F939D
:102290006F9385E492E09F938F938E010F5F1F4FA2
:1022A0001F930F930E9497330E9455266093210538
:1022B000709322058093230590932405B80180EF45
:1022C00095E00E94F82966ED72E080EF95E00E94AB
:1022D000F82987010FB6F894DEBF0FBECDBFE12C01
:1022E000F12CF80161918F0140E150E080EF95E021
:1022F0000E94032B60E673E080EF95E00E94F829CE
:10230000FFEFEF1AFF0A85E0E816F10451F765E5E3
:1023100072E080EF95E00E94F8298C8D811107C052
:102320006BE072E080EF95E00E94F82974C066E1EE
:1023300072E080EF95E00E94F82967E572E080EF97
:1023400095E00E94F8294AE050E0698980EF95E025
:102350000E94032B6BE572E080EF95E00E94F82964
:102360004AE050E06A8980EF95E00E94032B6CEA16
:1023700072E080EF95E00E94F8296B8970E04AE0F6
:1023800050E080EF95E00E94EE2A66EB72E080EF6D
:1023900095E00E94F8296C8970E04AE050E080EFF7
:1023A00095E00E94EE2A6EEB72E080EF95E00E94CD
:1023B000F8294D895E896F89788D22E030E080EFC1
:1023C00095E00E94FB2B65EC72E080EF95E00E94A7
:1023D000F829698D70E04AE050E080EF95E00E94B6
:1023E000EE2A60ED72E080EF95E00E94F8294AE065
:1023F00050E06A8D80EF95E00E94032B61E872E067
:1024000080EF95E00E94F8294AE050E06B8D80EF64
:1024100095E00E94032B80EF95E00E94012AA1968F
:102420000FB6F894DEBF0FBECDBFDF91CF911F91E5
:102430000F91FF90EF900895EF92FF920F931F93EB
:10244000CF93DF93CDB7DEB762970FB6F894DEBFB8
:102450000FBECDBF8C017B0161E673E00E947D2C35
:10246000F701808182958F708930D1F4BE016F5F52
:102470007F4FC7010E94C40F8C85882389F0BE015D
:102480006F5F7F4FCE010D960E945F10BE01635FAC
:102490007F4FC8010E94932CCE010D960E940F2CF5
:1024A000C80162960FB6F894DEBF0FBECDBFDF91B4
:1024B000CF911F910F91FF90EF9008951F93CF93AD
:1024C000DF9300D000D000D0CDB7DEB7BC01CE0185
:1024D00001960E941C128D819E81892B39F0BE01CC
:1024E0006F5F7F4F80EF95E00E94152A11E02D81EC
:1024F0003E81232B09F410E0CE0101960E940F2C9F
:10250000812F26960FB6F894DEBF0FBECDBFDF91A8
:10251000CF911F910895693523E4720781059105D4
:1025200049F021E06B3675428105910509F020E004
:10253000822F089581E0089565E00C94F11A8F923E
:102540009F92AF92BF92CF92DF92EF92FF920F9342
:102550001F93CF93DF938C01EB0181E08F87F8010C
:10256000F580FE86C8010E949C12F81659F08091F1
:102570002605882331F061EE72E080EF95E00E943D
:10258000272A1F86F80180818F7089838081829538
:102590008F7088838B3059F080912605882331F025
:1025A00060EF72E080EF95E00E94272A1F86F80115
:1025B000618162956F70F4E66F9FB00111248827E6
:1025C00077FD8095982F0E946D2E6B017C016A83A8
:1025D0007B838C839D83F80161816F70FAE06F9F2C
:1025E000B0011124882777FD8095982F0E946D2EC9
:1025F0009B01AC01C701B6010E946A2D6B017C01F1
:102600006A837B838C839D83F801628162956F70FE
:1026100070E080E090E00E946D2E9B01AC01C7014C
:10262000B6010E946A2D20E030E040E05FE30E94A6
:10263000212F6A837B838C839D83F80162816F7075
:10264000FAE06F9FB0011124882777FD8095982FBD
:102650000E946D2E6B017C016E837F838887998732
:10266000F801638162956F7070E080E090E00E94F5
:102670006D2E9B01AC01C701B6010E946A2D6B0152
:102680007C016E837F8388879987F80163816F70EF
:1026900070E080E090E00E946D2E2DEC3CEC4CEC64
:1026A0005DE30E94212F9B01AC01C701B6010E948E
:1026B0006A2D20E030E040E252E40E94692D6B0177
:1026C0007C016E837F8388879987F8016481629596
:1026D0006F7070E080E090E00E946D2E4B015C0115
:1026E0006A877B878C879D87F80164816F7070E0B3
:1026F00080E090E00E946D2E2DEC3CEC4CEC5DE314
:102700000E94212F9B01AC01C501B4010E946A2DDA
:102710006A877B878C879D8720E030E040E252EC1F
:10272000C701B6010E94CE2D87FD0AC020E030E02F
:1027300040E752E4C701B6010E941D2F1816ACF401
:102740001F8680912605882381F06FEF72E080EF6D
:1027500095E00E94F8294E815F816885798522E0A5
:1027600030E080EF95E00E94FD2BCA80DB80EC809A
:10277000FD8020E030E040E050E4C701B6010E9457
:10278000CE2D87FD0AC020E030E046E953E4C701C2
:10279000B6010E941D2F1816ACF41F8680912605E5
:1027A000882381F066E173E080EF95E00E94F829CC
:1027B0004A815B816C817D8122E030E080EF95E091
:1027C0000E94FD2BCA84DB84EC84FD8420E030E091
:1027D00040E050E4C701B6010E94CE2D87FD0AC03B
:1027E00020E030E040E551E4C701B6010E941D2F12
:1027F00018160CF51F86809126058823E1F067E204
:1028000073E080EF95E00E94F8294A855B856C852E
:102810007D8522E030E080EF95E0DF91CF911F9140
:102820000F91FF90EF90DF90CF90BF90AF909F906F
:102830008F900C94FD2BDF91CF911F910F91FF9002
:10284000EF90DF90CF90BF90AF909F908F900895C2
:10285000FF920F931F93CF93DF93EC018B0161E6FF
:1028600073E00E947D2C67E573E0CE010E94E62CA8
:10287000F8016181CE010E94092D6EE573E0CE0161
:102880000E94E62C20E030E040E251E4F801628151
:102890007381848195810E94212F20E030E04AE7F6
:1028A00054E40E946A2D0E943A2EF62E672FCE0124
:1028B0000E94092D60E673E0CE010E94E62C6F2D88
:1028C000CE010E94092D60E673E0CE010E94E62C45
:1028D00020E030E040E251E4F801668177818085B4
:1028E00091850E94212F20E030E04AE754E40E94C5
:1028F0006A2D0E943A2EF62E672FCE010E94092DD6
:1029000060E673E0CE010E94E62C6F2DCE010E949E
:10291000092D60E673E0CE010E94E62C20E030E055
:1029200040E251E4F80162857385848595850E94B3
:10293000212F0E943A2ECE010E94362DCE01DF912A
:10294000CF911F910F91FF900895EF92FF920F93F7
:102950001F93CF93DF93CDB7DEB766970FB6F8948A
:10296000DEBF0FBECDBF8C017B0161E673E00E942C
:102970007D2CBE016F5F7F4FC7010E949F12888927
:10298000882389F0BE016F5F7F4FCE0141960E9480
:102990002814BE016F5E7F4FC8010E94932CCE01A8
:1029A00041960E940F2CC80166960FB6F894DEBFC0
:1029B0000FBECDBFDF91CF911F910F91FF90EF9090
:1029C00008951F93CF93DF9300D000D000D0CDB7F0
:1029D000DEB7BC01CE0101960E94A5148D819E81B7
:1029E000892B39F0BE016F5F7F4F80EF95E00E9429
:1029F000152A11E02D813E81232B09F410E0CE0130
:102A000001960E940F2C812F26960FB6F894DEBFF8
:102A10000FBECDBFDF91CF911F9108956A3822E29A
:102A200072078105910579F06B3635E273078105F0
:102A3000910549F021E0693573448105910509F05C
:102A400020E0822F089581E00895FC01158A108A04
:102A5000FB0120E030E0DC01A20FB31F56964C9141
:102A600041932F5F3F4F20343105A9F70895FC01B2
:102A700085890895EF92FF921F93CF93DF931F9262
:102A8000CDB7DEB77C0118E0F701848190E0FC014E
:102A9000EA58FE4F2491FC01E657FE4F8491E82F3F
:102AA000F0E0EE0FFF1FE855FE4FA591B4918C9119
:102AB00090E0E22FF0E0E095F0958E239F238C9339
:102AC000F701828190E0FC01EA58FE4F67FF11C0D8
:102AD0002491FC01E657FE4F8491E82FF0E0EE0FC1
:102AE000FF1FE855FE4FA591B4918C91822B8C93DA
:102AF00016C04491FC01E657FE4F8491E82FF0E0A8
:102B0000EE0FFF1FE855FE4FA591B4912C9130E0D8
:102B1000E42FF0E0E095F0952E233F232C93660FF1
:102B2000F701848190E0FC01EA58FE4F2491FC01FA
:102B3000E657FE4FE491F0E0EE0FFF1FE855FE4F21
:102B4000A591B4918C91822B8C93F7018381698339
:102B50000E9489276981892B09F06160115009F071
:102B600093CFF701848190E0FC01EA58FE4F449135
:102B7000FC01E657FE4F8491E82FF0E0EE0FFF1FB7
:102B8000E855FE4FA591B4912C9130E0E42FF0E090
:102B9000E095F0952E233F232C93862F0F90DF9105
:102BA000CF911F91FF90EF900895FF920F931F9385
:102BB000CF93DF93EC018B0160E08D810E9453275E
:102BC00080E1F82E8A8190E0FC01EA58FE4F17FF61
:102BD00010C02491FC01E657FE4F8491E82FF0E0ED
:102BE000EE0FFF1FE855FE4FA591B4918C91822BFB
:102BF00015C02491FC01E657FE4F8491E82FF0E0C8
:102C0000EE0FFF1FE855FE4FA591B4918C9190E017
:102C1000E22FF0E0E095F0958E239F238C93000F38
:102C2000111F8B810E948927892B09F001608C81FB
:102C300090E0FC01EA58FE4F2491FC01E657FE4F5C
:102C4000E491F0E0EE0FFF1FE855FE4FA591B4911F
:102C50008C91822B8C9381E090E00E94AC268C8139
:102C600090E0FC01EA58FE4F2491FC01E657FE4F2C
:102C70008491E82FF0E0EE0FFF1FE855FE4FA5917D
:102C8000B4918C9190E0E22FF0E0E095F0958E23E6
:102C90009F238C93FA9409F095CF61E08D810E9477
:102CA0005327C801DF91CF911F910F91FF90089595
:102CB000CF93DF93EB010E94D51562E673E080EFBE
:102CC00095E00E94F8294AE050E0BE0180EF95E0CF
:102CD000DF91CF910C940A2B1F93CF93DF93EC01DC
:102CE000162F60E08D810E945327612F6F77CE01F0
:102CF0000E943A1560E0CE010E943A15182F61E05B
:102D00008D810E945327812FDF91CF911F910895CC
:102D1000FC01208131812230310519F460E00C94EE
:102D20006C1660E070EB0E94D51508950F931F9309
:102D3000CF93DF93EC01888199810297A9F468E22F
:102D4000CE010E946C1682FF48C000E010E0CE0168
:102D50000E948816FE01E00FF11F868B0F5F1F4F48
:102D600000341105A1F737C060E08D810E94532720
:102D7000000000008B810E9489278C0161E08D8119
:102D80000E945327012B89F0188981E0810F888BDD
:102D9000CE010E948816FE01E10FF11D868B0E9474
:102DA0005526698B7A8B8B8B9C8B8889811104C00B
:102DB0008889803280F411C00E94552609891A89B9
:102DC0002B893C890E5C1F4F2F4F3F4F061717076B
:102DD0002807390768F781E08D8BDF91CF911F912C
:102DE0000F910895EF92FF921F93CF93DF931F925D
:102DF000CDB7DEB77C01162F60E0FC0185814983E9
:102E00000E945327612F6068C7010E943A154981CB
:102E1000642FC7010E943A1561E0F70185810F9088
:102E2000DF91CF911F91FF90EF900C945327CF9299
:102E3000DF92EF92FF92CF93DF93EC019A01AB0107
:102E4000288739874A875B87888199810297F1F4BF
:102E5000CA01B9019695879577956795785B874103
:102E60009E4F0E94FD3069017A01432F552763E090
:102E7000CE010E94F2164C2D64E0CE01DF91CF917D
:102E8000FF90EF90DF90CF900C94F216CA01B90139
:102E90000E946B2E9B01AC0160E87FE588EA98E414
:102EA0000E94D22D6B017C0120E030E0A9010E943C
:102EB0001D2F20E030E040E05FE387FD05C0C70143
:102EC000B6010E946A2D04C0C701B6010E94692D97
:102ED0000E943A2E615070E0766CCE01DF91CF9166
:102EE000FF90EF90DF90CF900C94D515CF92DF92AA
:102EF000EF92FF92CF93DF93EC014C875D876E8753
:102F00007F87888199810297B1F5A8EEB3E09A0195
:102F1000AB010E944431A2E0660F771F881F991F02
:102F2000AA95D1F729E03DE340E050E00E94FD3052
:102F300069017A01B6E0CC0CDD1CEE1CFF1CBA95D1
:102F4000D1F7A7016627772767E0CE010E94F21626
:102F500077276F2D5E2D4D2D68E0CE010E94F21671
:102F60004C2D69E0CE01DF91CF91FF90EF90DF9083
:102F7000CF900C94F216CB01BA0160567F418D4080
:102F8000910925E030E040E050E00E94FD30B901B9
:102F90007056CE01DF91CF91FF90EF90DF90CF90F0
:102FA0000C94D515CF93DF93EC018881998166232A
:102FB00069F0029741F461E0CE010E946C16482F3F
:102FC000437E4C600CC068E372E811C0029769F45C
:102FD00061E0CE010E946C16482F437E446061E0A0
:102FE000CE01DF91CF910C94F21668E072E8CE0129
:102FF000DF91CF910C94D5151F93CF93DF93EC0104
:1030000088819981029741F440E168E2CE01DF9125
:10301000CF911F910C94F21610E460E070EBCE019A
:103020000E94D5151150C9F7DF91CF911F910895D6
:10303000CF93DF93EC01888199816623B9F00297E1
:1030400041F461E0CE010E946C16482F437E40613E
:1030500016C068EC72E8CE010E94D51561E87AECE2
:10306000CE010E94D51563E87AEC10C0029761F496
:1030700061E0CE010E946C16482F437E446061E0FF
:10308000CE010E94F21605C068E072E8CE010E94EF
:10309000D515CE01DF91CF910C94FC17CF93DF9320
:1030A000D62FC42F0E94F21669E673E080EF95E0F8
:1030B0000E94F8294AE050E06D2F80EF95E00E94D1
:1030C000032B63E773E080EF95E00E94F8294AE064
:1030D00050E06C2F80EF95E0DF91CF910C94032BA3
:1030E000FC01808191810895CF93DF93EC01FB0176
:1030F000808191818130910529F0029731F46CE74C
:1031000073E005C066E773E002C062E873E0CE01D9
:103110000E947D2CCE01DF91CF9108950F931F93D4
:10312000CF93DF9300D000D000D0CDB7DEB78C01B5
:10313000FC0187818823B1F067E873E080EF95E0B8
:103140000E94F829B801CE0101960E947418BE01B0
:103150006F5F7F4F80EF95E00E94152ACE010196A8
:103160000E940F2C61E0F80185810E94532760E0E6
:10317000C8010E941818F80180819181029709F016
:1031800056C044E061E0C8010E94F21640E062E0EF
:10319000C8010E94F21645E065E0C8010E94F216DF
:1031A00043EC66E0C8010E94F2164FE961E1C801F4
:1031B0000E94F2164FE063E1C8010E94F21642E459
:1031C00069E1C8010E94F21640E168E2C8010E946C
:1031D000F2164CED69E2C8010E94F21648E86EE270
:1031E000C8010E94F2164DE26FE2C8010E94F21679
:1031F00044ED60E3C8010E94F21648E067E3C801AD
:103200000E94F21640E468E3C8010E94F2164FE8FB
:103210006CE3C8010E94F21642E16DE3C8010E940E
:10322000F21640E36FE6C8010E94F2163CC068E067
:1032300072E8C8010E94D51568EE70E8C8010E94C6
:10324000D5156AE672ECC8010E94D51562E17AECE8
:10325000C8010E94D51564ED7EECC8010E94D51509
:1032600061E874ECC8010E94D51560EA74E9C801F0
:103270000E94D51567E77CECC8010E94D51560E572
:1032800078E9C8010E94D51560E070EEC8010E947F
:10329000D51560E078ECC8010E94D51560E470ECAB
:1032A000C8010E94D515F801448555856685778546
:1032B000C8010E947617F8014085518562857385A3
:1032C000C8010E941717C8010E94FC1726960FB666
:1032D000F894DEBF0FBECDBFDF91CF911F910F914C
:1032E0000895FC0181E020813181232B09F480E0E5
:1032F0000895CF92EF920F93CF93DF93EC01862F37
:103300006A834B832C830D83EE821F8249E553E44D
:1033100060E070E0488759876A877B874CEC5FE301
:103320006DE070E04C875D876E877F87188A198A09
:103330001A8A1B8A1C8A1D8A61E00E941A2760E093
:103340008B810E941A2761E08C810E941A2761E01C
:103350008D810E941A2761E08D810E945327198276
:1033600018824AE068E3CE010E94F21668E3CE01BB
:103370000E946C168A3079F440E468E3CE010E9422
:10338000F21668E3CE010E946C16803421F482E0CC
:1033900090E09983888388819981892B91F5C11068
:1033A0002CC06CE072E8CE010E94D51588EE93E047
:1033B00000000197E9F76FE470ECCE010E94D5158B
:1033C00088EE93E000000197E9F760E070E0CE013D
:1033D0000E94D51592FF15C060E470ECCE010E94EA
:1033E000D51588EE93E000000197E9F760E070E002
:1033F000CE010E94D51592FD04C081E090E0998332
:103400008883DF91CF910F91EF90CF900895FC01C9
:1034100067830895FC016085718582859385089591
:10342000FC01648575858685978508951F93CF93E4
:10343000DF93EC01162F60E070E0CE010E94D515FD
:1034400097FFF9CF612F70E0786BCE01DF91CF91BC
:103450001F910C94D5158F929F92AF92BF92DF92DD
:10346000EF92FF920F931F93CF93DF93EC017B01B9
:10347000D42E88819981029709F046C06DE3CE0170
:103480000E946C16482F44606DE3CE010E94F21634
:1034900060E0CE010E941818CE010E94FC17F8943B
:1034A00060E08D810E94532760E8CE010E943A15AA
:1034B000BE2C8701802F8B198D1538F4F80161918E
:1034C0008F01CE010E943A15F5CF61E08D810E94F7
:1034D0005327789461E0CE010E94D2170E945526AE
:1034E0004B015C0168E2CE010E946C1683FD3AC07C
:1034F0000E945526681979098A099B09643F714021
:103500008105910578F5EECF61E0CE010E94D217DA
:103510006AEACE010E94161A6AEACE010E94161AC1
:103520006AEACE010E94161A6DE2CE010E94161AB6
:1035300064EDCE010E94161A8701AD2CB12CC80192
:103540008E199F098A159B053CF4F80161918F0142
:10355000CE010E94161AF3CF61E070E080E090E0A7
:103560000E94842660E0CE010E94D2178F818823BA
:1035700061F162E973E080EF95E00E94F829E701CC
:103580000D2D10E0CE018E199F098017910774F45C
:1035900069914AE050E080EF95E00E94032B60E6DD
:1035A00073E080EF95E00E94F829ECCF80EF95E082
:1035B000DF91CF911F910F91FF90EF90DF90BF901F
:1035C000AF909F908F900C94012ADF91CF911F9123
:1035D0000F91FF90EF90DF90BF90AF909F908F90F2
:1035E0000895FC0140E070E0A1E39F01281B390B26
:1035F000261737076CF4519128E030E0B52FB42737
:10360000440FB7FD4A27550F21503109B9F7EDCFC7
:10361000842F0895809326050895FC0120E030E072
:1036200080E0A1E3919140E050E0BA01620F731F86
:103630006431710534F4692F6827880F67FD8A2784
:10364000990F4F5F5F4F4830510579F7285F3F4F23
:103650002831310539F70895FF920F931F93CF93C7
:10366000DF938C01EB0181E08B87F8018281F0E12F
:103670008F9FC0011124F801F380F294AFE0FA2289
:10368000F82AF986C8010E940D1BF8121B86F80162
:1036900080818F73898380818295869586958370DA
:1036A0008883833009F01B86F8019181892F881F58
:1036B0008827881F8A83818186FB882780F98B83EE
:1036C00061816F73F0E16F9FB0011124F801828175
:1036D00082958F70682B882777FD8095982F0E94A0
:1036E0006D2E2DEC3CEC4CEC5DE30E94212F20E094
:1036F00030E040E252E40E94692D6C837D838E832A
:103700009F83F80183818F708A878AE68887DF919B
:10371000CF911F910F91FF900895AF92BF92CF92DA
:10372000DF92EF92FF920F931F93CF93DF9300D01E
:1037300000D000D0CDB7DEB75C018B0161E673E04D
:10374000CE0101960E947D2C66EA72E0CE010196C0
:103750000E94E62CF8016181CE0101960E94092D9C
:1037600060E2CE0101960E94F62CF80180858F77E9
:10377000843610F08A3651F4F8018281882319F0DA
:1037800061E870E008C061E070E005C08D3709F0C5
:1037900042C062E870E0CE0101960E94362D60E2E0
:1037A000CE0101960E94F62C20E030E040E251E488
:1037B000F80164817581868197810E94212F20E024
:1037C00030E04AE754E40E946A2D0E943F2EF62E14
:1037D000672FCE0101960E94092D60E2CE0101966D
:1037E0000E94F62C6F2DCE0101960E94092D60E2F9
:1037F000CE0101960E94F62CF801C480D580E680A7
:10380000F78020E030E040E752E4C701B6010E94B3
:103810001D2F87FD06C061E673E0C5010E947D2C67
:1038200019C020E030E040E252ECC701B6010E942E
:10383000CE2D181684F7F8016085838181116068A8
:10384000CE0101960E94092DBE016F5F7F4FC50119
:103850000E94AA2CCE0101960E940F2CC50126962B
:103860000FB6F894DEBF0FBECDBFDF91CF911F9191
:103870000F91FF90EF90DF90CF90BF90AF900895A1
:10388000EF92FF920F931F93CF93DF93CDB7DEB7E5
:1038900062970FB6F894DEBF0FBECDBF8C017B01DF
:1038A00061E673E00E947D2CF7018081807C803C82
:1038B000D1F4BE016F5F7F4FC7010E942C1B8C8526
:1038C000882389F0BE016F5F7F4FCE010D960E9465
:1038D0008D1BBE01635F7F4FC8010E94932CCE01F8
:1038E0000D960E940F2CC80162960FB6F894DEBFA9
:1038F0000FBECDBFDF91CF911F910F91FF90EF9041
:1039000008951F93CF93DF9300D000D000D0CDB7A0
:10391000DEB7BC01CE0101960E94401C8D819E81C4
:10392000892B39F0BE016F5F7F4F80EF95E00E94D9
:10393000152A11E02D813E81232B09F410E0CE01E0
:1039400001960E940F2C812F26960FB6F894DEBFA9
:103950000FBECDBFDF91CF911F91089521E0693552
:1039600073448105910509F020E0822F089580912C
:10397000570590E020915805821B910908952091E8
:10398000580580915705281750F4E22FF0E0E75AC8
:10399000FA4F808190E02F5F2093580508958FEFB4
:1039A0009FEF0895E091580580915705E81730F48E
:1039B000F0E0E75AFA4F808190E008958FEF9FEF93
:1039C00008950895CF92DF92EF92FF920F931F9385
:1039D000CF93DF937C01CB018A0120913305222311
:1039E00089F0EB016B01C40ED51ECC15DD0569F025
:1039F0006991D701ED91FC910190F081E02DC70113
:103A00000995F3CF642F0E94431EC801DF91CF9127
:103A10001F910F91FF90EF90DF90CF900895CF937B
:103A2000DF931F92CDB7DEB7698320913305222340
:103A3000D1F020913405203240F021E030E0FC014B
:103A40003383228380E090E015C080913505E82F14
:103A5000F0E0EA5CFA4F998190838F5F809335059F
:103A60008093340505C061E0CE0101960E94431E9B
:103A700081E090E00F90DF91CF910895FC011382D7
:103A8000128248EE53E060E070E044835583668321
:103A900077838EEA93E0918380830895109258058E
:103AA0001092570510923505109234050C948E1D16
:103AB000862F413208F040E269E575E00E94AC1DB6
:103AC0001092580580935705089521E00C94581DD5
:103AD00081E080933305609356051092350510926E
:103AE000340508950C94681D0F93062F21E0409132
:103AF000340566E375E0809156050E94F01D109232
:103B0000350510923405109233050F91089561E048
:103B10000C94741D87E295E00C943E1D1092E6050E
:103B200081E08093E4051092E30561E082E10E9468
:103B3000532761E083E10E945327E9EBF0E08081A5
:103B40008E7F808380818D7F808388E48093B8001E
:103B500085E48093BC000895413208F03FC0909105
:103B6000E6059111FCCF91E09093E6052093E405E2
:103B70002FEF209379051092BE05240F2093BD05E9
:103B80009093E5059091E505880F892B8093E505D5
:103B90008091E305813041F41092E3058091E505C1
:103BA0008093BB0085EC01C085EE8093BC008091C2
:103BB000E6058130E1F38091BE05841710F4409151
:103BC000BE052FEB35E0FB01D9018A2F821B84173C
:103BD00018F48D918193F9CF842F089580E0089592
:103BE0000F93413208F046C09091E6059111FCCF49
:103BF00092E09093E6050093E4059FEF909379059A
:103C00001092BE054093BD05FB016FEB75E0DB0133
:103C10009A2F961B941718F491919D93F9CF1092B7
:103C2000E5059091E505880F892B8093E505809146
:103C3000E305813041F41092E3058091E50580931E
:103C4000BB0085EC01C085EE8093BC00222321F0EF
:103C50008091E6058230E1F3809179058F3F61F034
:103C600080917905803251F080917905803341F45B
:103C700083E007C081E005C080E003C082E001C0AE
:103C800084E00F910895613298F42091E605243084
:103C900089F460939B05FC018DE995E0DC012A2FF6
:103CA000281B261718F421912D93F9CF80E0089551
:103CB00081E0089582E0089585ED8093BC008091B5
:103CC000BC0084FDFCCF1092E605089585EC80933E
:103CD000BC001092E60508951F920F920FB60F9246
:103CE00011242F933F934F935F936F937F938F9301
:103CF0009F93AF93BF93EF93FF938091B900887F19
:103D0000803609F49CC068F5883209F45BC090F4F1
:103D1000803109F454C038F4882309F4F5C08830A0
:103D200009F44DC0F5C0883109F44CC0803209F463
:103D30005DC0EEC0803409F468C048F4803309F4F3
:103D400055C0883309F0E4C080937905A8C0803558
:103D500009F44FC0883509F45DC0883409F0D8C033
:103D6000D5C0883909F4C6C0A8F4883709F467C0FB
:103D700038F4883609F463C0803709F460C0C8C0DD
:103D8000883809F4B7C0803909F45FC0803809F079
:103D9000BFC05BC0803B09F485C038F4803A09F4A9
:103DA00066C0883A09F47EC0B3C0803C09F4A6C05E
:103DB000883C09F4A3C0883B09F489C0A9C080915C
:103DC000E50510C09091BE058091BD05981770F56E
:103DD000E091BE0581E08E0F8093BE05F0E0E154D6
:103DE000FA4F80818093BB0085EC85C08093790574
:103DF0008DC0E091BE0581E08E0F8093BE0580915D
:103E0000BB00F0E0E154FA4F80839091BE058091B1
:103E1000BD056DC0E091BE0581E08E0F8093BE05AB
:103E20008091BB00F0E0E154FA4F80838091E4057B
:103E300081116CC081E08093E30584EA60C083E077
:103E40008093E60510927A05CFCF80917A05803273
:103E500008F050C0E0917A0581E08E0F80937A05DA
:103E60008091BB00F0E0E558FA4F8083BDCF809190
:103E70007A05803230F4E0917A05F0E0E558FA4FA7
:103E800010820E945C1E60917A0570E0E091DF056F
:103E9000F091E0058BE795E0099510927A050E9474
:103EA000661E36C084E08093E60510929C05109251
:103EB0009B05E091E105F091E205099580919B0554
:103EC000811105C081E080939B0510929D05E091D2
:103ED0009C0581E08E0F80939C05F0E0E356FA4F3D
:103EE00080818093BB0090919C0580919B059817E1
:103EF00008F47ACF85E88093BC000AC085EC8093F3
:103F0000BC001092E60504C0109279050E945C1E68
:103F1000FF91EF91BF91AF919F918F917F916F91A1
:103F20005F914F913F912F910F900FBE0F901F9077
:103F30001895FC0181818770880F8D5F08952F92FD
:103F40003F924F925F926F927F928F929F92AF9229
:103F5000BF92CF92DF92EF92FF920F931F93CF9376
:103F6000DF93CDB7DEB763970FB6F894DEBF0FBE11
:103F7000CDBF8C010E94991F8150FE0139969E0190
:103F80002F5E3F4F1192E217F307E1F72889AF84C4
:103F9000CE848D849C84DB84EA84B984D801682F24
:103FA00070E091E0AD01401B510B461757070CF034
:103FB00078C08D91AE014F5F5F4FF22E20E030E070
:103FC000E82FE170E98BF82FF270FB8BE82FE4709B
:103FD0006E2EF82FF8705F2EE82FE0714E2EF82F1E
:103FE000F0723F2EE82FE0742E2EF9013197E73062
:103FF000F10520F4E759FF4F0C943E31E82FEE0F06
:10400000EE0BE923E9832BC0222011F09A8327C00D
:104010001A8225C0332011F09B8321C01B821FC050
:10402000442011F09C831BC01C8219C0552011F044
:104030009D8315C01D8213C0662011F09E830FC0A2
:104040001E820DC0FB89FF2311F09F8308C01F82D1
:1040500006C07988772011F0988701C01886FA0188
:104060007190AF017A8AE72DE13009F4F724F82D39
:10407000FF25892C8F242F5F3F4F2830310549F0D1
:10408000EA2DAC2CCF2E9D2CDE2CEB2CBF2CFE2E43
:10409000ACCF2A2DAC2CCF2E9D2CDE2CEB2CBF2CA4
:1040A00081CFF0E82F9F9001112440E4A49EC0012D
:1040B0001124822B8B2990E2C99E90011124822B1E
:1040C000E0E18E9E90011124822BF8E09F9E9001EA
:1040D0001124822B44E0D49E90011124822BEE0CFB
:1040E0008E2963960FB6F894DEBF0FBECDBFDF9169
:1040F000CF911F910F91FF90EF90DF90CF90BF90E5
:10410000AF909F908F907F906F905F904F903F9077
:104110002F9008957F928F929F92AF92BF92CF92ED
:10412000DF92EF92FF920F931F93CF93DF938C0157
:10413000EB0181E08E83188219821A821B821C8215
:104140001F82188619861A861B861C861D861E8667
:104150001F86188A198A1A8A1B8A1C8A1D8A1E8A37
:104160001F8A188E198E1A8E1B8E1C8E1D8E1E8E07
:104170001F8E18A219A21D82C8010E94991FF80162
:10418000E80FF11D3197F080FD82C8010E949F1F4A
:10419000F8121E82F801808182958F7088838A30A0
:1041A00009F01E828E81882309F4E6C0F80180811F
:1041B0008F70F4E08F9FC0011124F80191819295D6
:1041C000969596959370982B9983918181E095FFB0
:1041D00080E08A83F801918181E094FF80E08C8304
:1041E000F80181818F7083FB882780F98B8381811F
:1041F00087700D5F1F4FE12CF12CC82ED12C772436
:104200007394EC14FD040CF0B7C0FFEFEF1AFF0A33
:10421000F80131979081F8016081892F8F70B62E57
:10422000B2942FE0B2226F70A62E92959F709230BA
:1042300009F45CC030F4992311F1913009F449C0BC
:1042400098C0933009F46CC0943009F092C07C8619
:1042500070E080E1B89E600D711D1124882777FD04
:104260008095982F0E946D2E20E030E040E251E4CE
:104270000E94D22D6E8F7F8F88A399A37AC07F82F0
:10428000462F6B2D0E94E92420E030E048EC53E4F7
:104290000E94692D20E030E040E251E40E94D22DDE
:1042A0004B015C016D877E878F87988B20E030E023
:1042B00040E752E40E941D2F1816B4F020E030E0D1
:1042C00040E252ECC501B4010E94CE2D87FF51C0DF
:1042D0000BC09887462F6B2D0E94E9240E943F2E29
:1042E000698B653608F445C01E8243C079866B2D04
:1042F00070E0F0E18F9F600D711D112484E0660F66
:10430000771F8A95E1F76A0D711D882777FD8095E3
:10431000982F0E946D2E6A8B7B8B8C8B9D8B29C076
:104320007B867A86682F70E080E090E00E946D2E98
:1043300020E030E044EB51E40E94212F6E8B7F8B14
:10434000888F998F6A2D70E020E1B29E600D711DFB
:104350001124882777FD8095982F0E946D2E20E0EC
:1043600030E040E251E40E94D22D6A8F7B8F8C8F27
:104370009D8F0E5F1F4F45CFDF91CF911F910F9102
:10438000FF90EF90DF90CF90BF90AF909F908F9075
:104390007F900895EF92FF920F931F93CF93DF9337
:1043A000CDB7DEB7A8970FB6F894DEBF0FBECDBF6E
:1043B0008C017B0161E673E00E947D2CF701808116
:1043C000807A803AD9F4BE016F5F7F4FC7010E94A7
:1043D0008A208F81882391F041E0BE016F5F7F4F7B
:1043E000CE0183960E94C423BE016D5D7F4FC8013C
:1043F0000E94932CCE0183960E940F2CC801A89690
:104400000FB6F894DEBF0FBECDBFDF91CF911F91E5
:104410000F91FF90EF9008951F93CF93DF9300D0FB
:1044200000D000D0CDB7DEB7BC01CE0101960E940E
:10443000CA218D819E81892B39F0BE016F5F7F4F2C
:1044400080EF95E00E94152A11E02D813E81232BFB
:1044500009F410E0CE0101960E940F2C812F2696C0
:104460000FB6F894DEBF0FBECDBFDF91CF911F9185
:10447000089521E06A3872428105910509F020E033
:10448000822F089569E00C94F11AFF920F931F9305
:10449000CF93DF938C01EB0181E08E8319821A8226
:1044A0001B821C828F83888789878A878B878C876A
:1044B000F801F184FD82C8010E944222F8121E8296
:1044C000F801808190E024E0959587952A95E1F7A1
:1044D00088838A3009F01E828E81882309F47BC08C
:1044E000F8018081F0E18F9FC0011124F8019181D2
:1044F00092959F70982B99831A821C821B828181CE
:10450000682F677070E0762F66279281692B83FF92
:1045100003C0719561957109882777FD8095982F63
:104520000E946D2E2DEC3CEC4CEC5DE30E94212FA3
:104530006D877E878F87988BF80183818F77898B32
:10454000648170E080E090E00E946D2E2BE734E102
:104550004EEA5EE30E94212F6A8F7B8F8C8F9D8FA6
:10456000F801658170E080E090E00E946D2E2BE7FD
:1045700034E14EEA5EE30E94212F6E8F7F8F88A385
:1045800099A3F80166816F7070E0762F66278781A6
:10459000682B882777FD8095982F0E946D2E2AE939
:1045A00039E949E15FE30E94212F6A8B7B8B8C8B79
:1045B0009D8BF80160856F7070E080E090E00E9454
:1045C0006D2E20E030E044EB51E40E94212F6E8BF1
:1045D0007F8B888F998FDF91CF911F910F91FF90E3
:1045E0000895EF92FF920F931F93CF93DF93CDB770
:1045F000DEB7A8970FB6F894DEBF0FBECDBF8C0113
:104600007B0161E673E00E947D2CF701208130E0A0
:1046100044E0359527954A95E1F72A303105D9F4DC
:10462000BE016F5F7F4FC7010E9445228F818823A3
:1046300091F043E0BE016F5F7F4FCE0183960E94F1
:10464000C423BE016D5D7F4FC8010E94932CCE0133
:1046500083960E940F2CC801A8960FB6F894DEBF6F
:104660000FBECDBFDF91CF911F910F91FF90EF90C3
:1046700008951F93CF93DF9300D000D000D0CDB723
:10468000DEB7BC01CE0101960E94F1228D819E8190
:10469000892B39F0BE016F5F7F4F80EF95E00E945C
:1046A000152A11E02D813E81232B09F410E0CE0163
:1046B00001960E940F2C812F26960FB6F894DEBF2C
:1046C0000FBECDBFDF91CF911F91089521E06935D5
:1046D00073448105910509F020E0822F0895EF923F
:1046E000FF920F931F93CF93DF931F92CDB7DEB747
:1046F0007C01162F072F61E673E049830E947D2C11
:104700004981411102C01FEF0FEF60E2C7010E9413
:10471000F62C602FC7010E94092D60E2C7010E949C
:10472000F62C612FC7010E94092DC7010F90DF9160
:10473000CF911F910F91FF90EF900895EF92FF920C
:104740001F93CF93DF931F92CDB7DEB77C01162F57
:1047500061E673E049830E947D2C60E2C7010E94FC
:10476000F62C4981442319F0612F70E002C06FEFED
:1047700070E0C7010E94362DC7010F90DF91CF91E5
:104780001F91FF90EF9008958F929F92AF92BF92EA
:10479000CF92DF92EF92FF920F931F93CF93DF930D
:1047A00000D000D000D0CDB7DEB75C018B01842EE5
:1047B00061E673E00E947D2CF801948081E09826E8
:1047C00087818823C9F0C584D684E784F08820E0F7
:1047D00030E040E252ECC701B6010E94CE2D87FDC9
:1047E0000AC02AE939E94FE652E4C701B6010E943E
:1047F0001D2F18160CF4912CF8018085882329F0C0
:1048000081898150833608F0D0C0992009F4CDC049
:1048100063E972E0C5010E94E62CF8016181C501DF
:104820000E94092D60E673E0C5010E94E62C682D08
:10483000C5010E94092D20E030E040E251E4F8017A
:1048400065857685878590890E94212F20E030E05C
:104850004AE754E40E946A2D0E943F2EF8014781E6
:10486000CE0101960E946F23BE016F5F7F4FC5018D
:104870000E94DF2CCE0101960E940F2CF80140858A
:104880006189CE0101960E949E23BE016F5F7F4F1A
:10489000C5010E94DF2CCE0101960E940F2CF80169
:1048A00062897389848995890E943F2EF801418528
:1048B000CE0101960E946F23BE016F5F7F4FC5013D
:1048C0000E94DF2CCE0101960E940F2C20E030E0E8
:1048D00040E251E4F80166897789808D918D0E94CC
:1048E000212F0E943F2EF8014385CE0101960E94A0
:1048F0006F23BE016F5F7F4FC5010E94DF2CCE0189
:1049000001960E940F2C20E030E040E251E4F801D3
:10491000628D738D848D958D0E94212F0E943F2E74
:10492000F8014285CE0101960E946F23BE016F5FA0
:104930007F4FC5010E94DF2CCE0101960E940F2CF3
:1049400020E030E040E251E4F801668D778D80A1EF
:1049500091A10E94212F0E943F2EF8014485CE0193
:1049600001960E946F23BE016F5F7F4FC5010E94B9
:10497000DF2CCE0101960E940F2CF8016281848108
:1049800081116E5FF801838181116C5F41E0CE017E
:1049900001960E949E23BE016F5F7F4FC5010E945A
:1049A000DF2CCE0101960E940F2CC50126960FB672
:1049B000F894DEBF0FBECDBFDF91CF911F910F9155
:1049C000FF90EF90DF90CF90BF90AF909F908F902F
:1049D0000895CF92DF92EF92FF92CF93DF93D62F7D
:1049E000C42F24E6829FC0011124BC01882777FDD3
:1049F0008095982F0E946D2E20E030E0A9010E9442
:104A00006A2D6B017C018AE0D89FB00111248827B0
:104A100077FD8095982F0E946D2E9B01AC01C701F8
:104A2000B6010E946A2D6B017C016C2F70E080E062
:104A300090E00E946D2E9B01AC01C701B6010E945F
:104A40006A2DDF91CF91FF90EF90DF90CF90089586
:104A500020E030E040E0FC015191CF01450F2F5F95
:104A60003F4F26303105B9F781E0411180E00895CC
:104A7000CF92DF92EF92FF920F931F93CF93DF932A
:104A80008C01EB0181E08B87F8018081888385812F
:104A90008A87C8010E9428258B87F8019181292FD8
:104AA0002F70907392959F7009F494E0F0E19F9FAE
:104AB000C0011124822B8983F801628170E0625366
:104AC0007109882777FD8095982F0E946D2E20E030
:104AD00030E040E251E40E94212F6B017C01F8019B
:104AE000638170E080E090E00E946D2E9B01AC013C
:104AF000C701B6010E946A2D20E030E040E251E497
:104B00000E94D22D6C837D838E839F83F8018481E4
:104B10008987818190E026E0959587952A95E1F730
:104B200021E0892B09F420E02887DF91CF911F91A4
:104B30000F91FF90EF90DF90CF900895EF92FF924A
:104B40000F931F93CF93DF93CDB7DEB762970FB666
:104B5000F894DEBF0FBECDBF8C017B0161E673E030
:104B60000E947D2CF70180818135D1F4BE016F5FF9
:104B70007F4FC7010E9438258C85882389F0BE01AC
:104B80006F5F7F4FCE010D960E945F10BE01635F85
:104B90007F4FC8010E94932CCE010D960E940F2CCE
:104BA000C80162960FB6F894DEBF0FBECDBFDF918D
:104BB000CF911F910F91FF90EF9008951F93CF9386
:104BC000DF9300D000D000D0CDB7DEB7BC01CE015E
:104BD00001960E949E258D819E81892B39F0BE0110
:104BE0006F5F7F4F80EF95E00E94152A11E02D81C5
:104BF0003E81232B09F410E0CE0101960E940F2C78
:104C0000812F26960FB6F894DEBF0FBECDBFDF9181
:104C1000CF911F9108951F920F920FB60F921124FA
:104C20002F933F938F939F93AF93BF938091E8050A
:104C30009091E905A091EA05B091EB053091E70567
:104C400023E0230F2D3720F40196A11DB11D05C0CF
:104C500026E8230F0296A11DB11D2093E70580933E
:104C6000E8059093E905A093EA05B093EB058091E0
:104C7000EC059091ED05A091EE05B091EF05019640
:104C8000A11DB11D8093EC059093ED05A093EE0559
:104C9000B093EF05BF91AF919F918F913F912F916D
:104CA0000F900FBE0F901F9018952FB7F89460913A
:104CB000E8057091E9058091EA059091EB052FBF19
:104CC00008953FB7F8948091EC059091ED05A0917F
:104CD000EE05B091EF0526B5A89B05C02F3F19F052
:104CE0000196A11DB11D3FBF6627782F892F9A2FEE
:104CF000620F711D811D911D42E0660F771F881F95
:104D0000991F4A95D1F70895CF92DF92EF92FF92C3
:104D1000CF93DF936B017C010E946126EB01C114EC
:104D2000D104E104F10489F00E94682D0E946126FB
:104D30006C1B7D0B683E734090F381E0C81AD1086C
:104D4000E108F108C851DC4FEACFDF91CF91FF9025
:104D5000EF90DF90CF900895019739F0880F991F59
:104D6000880F991F02970197F1F70895789484B5F9
:104D7000826084BD84B5816084BD85B5826085BD57
:104D800085B5816085BDEEE6F0E08081816080833D
:104D9000E1E8F0E010828081826080838081816020
:104DA0008083E0E8F0E0808181608083E1EBF0E0E7
:104DB000808184608083E0EBF0E08081816080838B
:104DC000EAE7F0E080818460808380818260808374
:104DD0008081816080838081806880831092C1009F
:104DE0000895833081F028F4813099F08230A1F069
:104DF00008958730A9F08830B9F08430D1F48091DB
:104E000080008F7D03C0809180008F778093800029
:104E1000089584B58F7702C084B58F7D84BD0895D1
:104E20008091B0008F7703C08091B0008F7D809318
:104E3000B0000895CF93DF9390E0FC01EA58FE4F55
:104E40002491FC01E657FE4F8491882349F190E0BC
:104E5000880F991FFC01EE54FE4FA591B49188551F
:104E60009E4FFC01C591D4919FB7611108C0F89481
:104E70008C91209582238C93888182230AC0623092
:104E800051F4F8948C91322F309583238C93888140
:104E9000822B888304C0F8948C91822B8C939FBFC3
:104EA000DF91CF9108950F931F93CF93DF931F92BC
:104EB000CDB7DEB7282F30E0F901EE59FE4F8491CF
:104EC000F901EA58FE4F1491F901E657FE4F04919B
:104ED0000023C9F0882321F069830E94F1266981AB
:104EE000E02FF0E0EE0FFF1FE855FE4FA591B491C3
:104EF0009FB7F8948C91611103C01095812301C074
:104F0000812B8C939FBF0F90DF91CF911F910F91B9
:104F10000895CF93DF93282F30E0F901EE59FE4F2B
:104F20008491F901EA58FE4FD491F901E657FE4FFA
:104F3000C491CC2391F081110E94F126EC2FF0E076
:104F4000EE0FFF1FE256FE4FA591B4912C912D2339
:104F500081E090E021F480E002C080E090E0DF9109
:104F6000CF910895FC01818D228D90E0805C9F4F50
:104F7000821B91098F7399270895FC01918D828D71
:104F8000981731F0828DE80FF11D858D90E008951E
:104F90008FEF9FEF0895FC01918D828D981761F03E
:104FA000828DDF01A80FB11D5D968C91928D9F5F60
:104FB0009F73928F90E008958FEF9FEF08958FE495
:104FC00099E2892B49F080E090E0892B29F00E943A
:104FD0004F2981110C9400000895FC01848DDF019C
:104FE000A80FB11DA35ABF4F2C91848D90E001965C
:104FF0008F739927848FA689B7892C93A089B1894B
:105000008C9180648C93938D848D981306C0028854
:10501000F389E02D80818F7D80830895CF93DF9386
:10502000EC01888D8823C9F0EA89FB89808185FDA0
:1050300005C0A889B9898C9186FD0FC00FB607FC01
:10504000F5CF808185FFF2CFA889B9898C9185FF42
:10505000EDCFCE010E94ED27E7CFDF91CF910895EC
:10506000CF92DF92FF920F931F93CF93DF931F9204
:10507000CDB7DEB76C01DC015B969C915B975C96CB
:105080008C915C97981307C05096ED91FC915197C5
:10509000808185FD32C0F601038D10E00F5F1F4F48
:1050A0000F731127F02EF601848DF81211C00FB680
:1050B00007FCF9CFD6015096ED91FC915197808174
:1050C00085FFF1CFC60169830E94ED276981EBCF8F
:1050D000838DE80FF11DE35AFF4F6083D6015B9685
:1050E0000C935B975296ED91FC915397808180626F
:1050F000808381E058968C930DC0D6015696ED9131
:10510000FC91579760835096ED91FC915197808167
:105110008064808381E090E00F90DF91CF911F91B8
:105120000F91FF90DF90CF900895BF92CF92DF92C2
:10513000EF92FF92CF93DF93EC016A017B01B22ED5
:10514000E889F98982E08083411581EE580761057D
:105150007105A1F060E079E08DE390E0A701960190
:105160000E94FD302150310941095109569547955A
:1051700037952795211580E1380798F0E889F98956
:10518000108260E874E88EE190E0A70196010E9429
:10519000FD30215031094109510956954795379500
:1051A0002795EC85FD853083EE85FF852083188E5D
:1051B000EC89FD89B082EA89FB89808180618083E6
:1051C000EA89FB89808188608083EA89FB89808104
:1051D00080688083EA89FB8980818F7D8083DF916D
:1051E000CF91FF90EF90DF90CF90BF9008951F92E6
:1051F0000F920FB60F9211242F938F939F93EF93DB
:10520000FF93E0910006F09101068081E09106068F
:10521000F091070682FD12C09081809109068F5F90
:105220008F7320910A06821751F0E0910906F0E091
:10523000E051FA4F958F8093090601C08081FF915C
:10524000EF919F918F912F910F900FBE0F901F9014
:1052500018951F920F920FB60F9211242F933F9320
:105260004F935F936F937F938F939F93AF93BF936E
:10527000EF93FF9380EF95E00E94ED27FF91EF9170
:10528000BF91AF919F918F917F916F915F914F915E
:105290003F912F910F900FBE0F901F90189580EFA8
:1052A00095E00E94B22721E0892B09F420E0822FAB
:1052B00008951092F3051092F20588EE93E0A0E0B5
:1052C000B0E08093F4059093F505A093F605B093B4
:1052D000F70583E094E09093F1058093F00585EC69
:1052E00090E09093FD058093FC0584EC90E0909312
:1052F000FF058093FE0580EC90E09093010680937B
:10530000000681EC90E0909303068093020682EC05
:1053100090E0909305068093040686EC90E09093CD
:105320000706809306061092090610920A0610924C
:105330000B0610920C06089508950E94B6260E944E
:105340009C290E94BF04CFEDD7E20E9478052097E8
:10535000E1F30E94DF27F9CFCF92DF92EF92FF9225
:105360000F931F93CF93DF936C017A01EB01E60E4D
:10537000F71E00E010E0CE15DF0561F06991D6015F
:10538000ED91FC910190F081E02DC6010995080F87
:10539000191FF1CFC801DF91CF911F910F91FF909D
:1053A000EF90DF90CF9008956115710581F0DB01DA
:1053B0000D900020E9F7AD0141505109461B570BF4
:1053C000DC01ED91FC910280F381E02D099480E0F5
:1053D00090E00895DC01ED91FC91DB0114964D9174
:1053E0005C9115976D917C910280F381E02D099479
:1053F0000C94D429DC01ED91FC910190F081E02D19
:1054000009940F931F93CF93DF93EC016DE00E94FB
:10541000FA298C016AE0CE010E94FA29800F911FBF
:10542000DF91CF911F910F9108950F931F93CF9309
:10543000DF93EC010E94EA298C01CE010E94012A2F
:10544000800F911FDF91CF911F910F9108950F93BE
:105450001F93CF93DF93EC010E94D4298C01CE01DE
:105460000E94012A800F911FDF91CF911F910F9110
:1054700008950F931F93CF93DF93EC010E94FA29B5
:105480008C01CE010E94012A800F911FDF91CF91E4
:105490001F910F9108958F929F92AF92BF92CF92DA
:1054A000DF92EF92FF920F931F93CF93DF93CDB7CD
:1054B000DEB7A1970FB6F894DEBF0FBECDBF7C015B
:1054C000C42EE52FCB01D22E19A221E02D1510F00C
:1054D0002AE0D22E8E010F5D1F4F8D2C912CA12C16
:1054E000B12C6C2D7E2FA50194010E94FD308C2DD6
:1054F000D29E80191124015011098A3014F4805D64
:1055000001C0895CF80180832115310541055105F1
:1055100021F0C22EE32FCA01E4CFB801C7010E94D7
:10552000D429A1960FB6F894DEBF0FBECDBFDF9190
:10553000CF911F910F91FF90EF90DF90CF90BF9090
:10554000AF909F908F900895CF92DF92EF92FF924D
:105550000F931F93CF93DF93EC016A017B01211519
:10556000310579F4E881F9810190F081E02D642F13
:10557000DF91CF911F910F91FF90EF90DF90CF902F
:1055800009942A303105E9F477FF1AC06DE20E94D0
:10559000FA298C0144275527BA014C195D096E0977
:1055A0007F092AE0CE010E944B2A800F911FDF91D4
:1055B000CF911F910F91FF90EF90DF90CF900895C2
:1055C0002AE0B701A601CE01DF91CF911F910F9183
:1055D000FF90EF90DF90CF900C944B2A9A01AB0193
:1055E000662757FD6095762F0C94A42A2115310566
:1055F00041F4DC01ED91FC910190F081E02D642FEC
:1056000009940C944B2A9A01462F50E060E070E018
:105610000C94F62A9A01AB0160E070E00C94F62A33
:105620004F925F926F927F928F929F92AF92BF92B2
:10563000CF92DF92EF92FF920F931F93CF93DF935E
:10564000EC016A017B01B22E9A01AB01C701B601E0
:105650000E94D02F882319F06FE074E027C0260144
:105660003701E89477F82FEF3FEF4FE75FE7C3018B
:10567000B2010E94D02F81110DC02FEF3FEF4FE7F5
:105680005FE7C301B2010E94CE2D18161CF463E13E
:1056900074E00CC02FEF3FEF4FE75FE4C701B601A6
:1056A0000E941D2F1816ACF467E174E0CE01DF9163
:1056B000CF911F910F91FF90EF90DF90CF90BF900F
:1056C000AF909F908F907F906F905F904F900C94D1
:1056D000D4292FEF3FEF4FE75FECC701B6010E94DF
:1056E000CE2D87FDE1CF20E030E0A901C701B60152
:1056F0000E94CE2D87FF0AC06DE2CE010E94FA29DA
:105700008C01F7FAF094F7F8F09402C000E010E092
:10571000A12C60E070E080E09FE3AB1441F020E05A
:1057200030E040E251E40E94D22DA394F6CF9B01D9
:10573000AC01C701B6010E946A2D6B017C010E9479
:105740003F2E2B013C010E946B2E9B01AC01C70137
:10575000B6010E94692D6B017C012AE0B301A20110
:10576000CE010E944B2A080F191FBB2039F06BE1B4
:1057700074E0CE010E94D429080F191F7B2C7720DA
:1057800041F120E030E040E251E4C701B6010E945F
:10579000212F6B017C010E943A2E4B01AA2497FC19
:1057A000A094BA2C2AE030E0B501A401CE010E94F9
:1057B000A42A080F191FC501B4010E946D2E9B0178
:1057C000AC01C701B6010E94692D6B017C017A947E
:1057D000D6CFC801DF91CF911F910F91FF90EF902D
:1057E000DF90CF90BF90AF909F908F907F906F9001
:1057F0005F904F9008950C94102B0F931F93CF93AD
:10580000DF93EC010E94102B8C01CE010E94012A33
:10581000800F911FDF91CF911F910F910895FC018F
:10582000808191810C94FE31CF93DF93EC018881CC
:105830009981009711F00E94FE31198218821D8211
:105840001C821B821A82DF91CF9108950F931F93C0
:10585000CF93DF93EC018B016F5F7F4F888199813C
:105860000E948D32009731F0998388831B830A83CD
:1058700081E001C080E0DF91CF911F910F910895E9
:10588000CF93DF93EC0188819981892B29F08A815C
:105890009B818617970760F4CE010E94262C8823EF
:1058A00041F08C819D81892B19F4E881F981108266
:1058B00081E0DF91CF910895EF92FF920F931F93B4
:1058C000CF93DF93EC017B018A01BA010E94402C47
:1058D000811104C0CE010E94142C07C01D830C83CB
:1058E000B701888199810E946033CE01DF91CF9109
:1058F0001F910F91FF90EF900895FC01118210828B
:1059000013821282158214826115710559F0FB0110
:1059100001900020E9F7AF0141505109461B570B98
:105920000C945C2C0895CF93DF93EC01FB01861758
:10593000970761F0608171816115710529F04481DB
:1059400055810E945C2C02C00E94142CCE01DF9174
:10595000CF910895FC011182108213821282158268
:1059600014820C94932CEF92FF920F931F93CF937A
:10597000DF93EC017B010C811D816115710511F430
:1059800080E016C04115510591F0040F151FB801B4
:105990000E94402C8823A1F3288139818C819D812C
:1059A000B701820F931F0E9460331D830C8381E037
:1059B000DF91CF911F910F91FF90EF900895FB0120
:1059C00044815581608171810C94B32C61157105FE
:1059D00059F0FB0101900020E9F7AF014150510956
:1059E000461B570B0C94B32C80E00895CF93DF93A4
:1059F00000D0CDB7DEB769831A8241E050E0BE0126
:105A00006F5F7F4F0E94B32C0F900F90DF91CF916B
:105A10000895EF92FF920F931F93CF93DF9300D0DF
:105A200000D0CDB7DEB77C01862F4AE050E08E0172
:105A30000F5F1F4FB80190E00E946733F80101909B
:105A40000020E9F7AF0141505109401B510BB8014B
:105A5000C7010E94B32C0F900F900F900F90DF9111
:105A6000CF911F910F91FF90EF900895EF92FF92C9
:105A70000F931F93CF93DF93CDB7DEB728970FB661
:105A8000F894DEBF0FBECDBF7C01CB014AE050E0F1
:105A90008E010F5F1F4FB8010E946733F80101901C
:105AA0000020E9F7AF0141505109401B510BB801EB
:105AB000C7010E94B32C28960FB6F894DEBF0FBE24
:105AC000CDBFDF91CF911F910F91FF90EF9008957F
:105AD00008955058BB27AA270ED075C166D130F063
:105AE0006BD120F031F49F3F11F41EF45BC10EF432
:105AF000E095E7FB51C1E92F77D180F3BA17620730
:105B000073078407950718F071F49EF58FC10EF4A2
:105B1000E0950B2EBA2FA02D0B01B90190010C01BD
:105B2000CA01A0011124FF27591B99F0593F50F4D5
:105B3000503E68F11A16F040A22F232F342F44272D
:105B4000585FF3CF469537952795A795F040539525
:105B5000C9F77EF41F16BA0B620B730B840BBAF0F5
:105B60009150A1F0FF0FBB1F661F771F881FC2F760
:105B70000EC0BA0F621F731F841F48F48795779574
:105B80006795B795F7959E3F08F0B3CF9395880F2B
:105B900008F09927EE0F979587950895D9D008F4C6
:105BA00081E008950CD00FC107D140F0FED030F055
:105BB00021F45F3F19F0F0C0511139C1F3C014D185
:105BC00098F39923C9F35523B1F3951B550BBB27C4
:105BD000AA2762177307840738F09F5F5F4F220F71
:105BE000331F441FAA1FA9F333D00E2E3AF0E0E86A
:105BF00030D091505040E695001CCAF729D0FE2FB6
:105C000027D0660F771F881FBB1F26173707480747
:105C1000AB07B0E809F0BB0B802DBF01FF279358FD
:105C20005F4F2AF09E3F510568F0B6C000C15F3F4C
:105C3000ECF3983EDCF3869577956795B795F795E5
:105C40009F5FC9F7880F911D9695879597F90895DD
:105C5000E1E0660F771F881FBB1F62177307840779
:105C6000BA0720F0621B730B840BBA0BEE1F88F788
:105C7000E095089504D06894B111D9C00895BCD0BE
:105C800088F09F5790F0B92F9927B751A0F0D1F025
:105C9000660F771F881F991F1AF0BA95C9F712C0AF
:105CA000B13081F0C3D0B1E00895C0C0672F782F24
:105CB0008827B85F39F0B93FCCF38695779567951B
:105CC000B395D9F73EF490958095709561957F4F87
:105CD0008F4F9F4F0895E89409C097FB3EF490952D
:105CE0008095709561957F4F8F4F9F4F9923A9F0B5
:105CF000F92F96E9BB279395F69587957795679544
:105D0000B795F111F8CFFAF4BB0F11F460FF1BC087
:105D10006F5F7F4F8F4F9F4F16C0882311F096E91A
:105D200011C0772321F09EE8872F762F05C06623C8
:105D300071F096E8862F70E060E02AF09A95660F81
:105D4000771F881FDAF7880F9695879597F908953A
:105D5000990F0008550FAA0BE0E8FEEF161617067C
:105D6000E807F907C0F012161306E407F50798F0E4
:105D7000621B730B840B950B39F40A2661F0232BFD
:105D8000242B252B21F408950A2609F4A140A69579
:105D90008FEF811D811D089597F99F6780E870E05E
:105DA00060E008959FEF80EC089500240A94161691
:105DB000170618060906089500240A9412161306F9
:105DC000140605060895092E0394000C11F4882387
:105DD00052F0BB0F40F4BF2B11F460FF04C06F5FA3
:105DE0007F4F8F4F9F4F089557FD9058440F551F79
:105DF00059F05F3F71F04795880F97FB991F61F04D
:105E00009F3F79F087950895121613061406551FC3
:105E1000F2CF4695F1DF08C0161617061806991F2F
:105E2000F1CF86957105610508940895E894BB2724
:105E300066277727CB0197F908958ADF08F48FEF5B
:105E400008950BD0C0CFB1DF28F0B6DF18F095234E
:105E500009F0A2CFA7CF1124EACFC6DFA0F3959F08
:105E6000D1F3950F50E0551F629FF001729FBB2741
:105E7000F00DB11D639FAA27F00DB11DAA1F649FED
:105E80006627B00DA11D661F829F2227B00DA11DA0
:105E9000621F739FB00DA11D621F839FA00D611D26
:105EA000221F749F3327A00D611D231F849F600D47
:105EB000211D822F762F6A2F11249F5750408AF080
:105EC000E1F088234AF0EE0FFF1FBB1F661F771F0C
:105ED000881F91505040A9F79E3F510570F05CCF4C
:105EE000A6CF5F3FECF3983EDCF3869577956795F8
:105EF000B795F795E7959F5FC1F7FE2B880F911D2A
:105F00009695879597F90895FA01EE0FFF1F309641
:105F10002105310599F16115710561F48038BFE300
:105F20009B0749F168949038810561F08038BFEF94
:105F30009B0741F0992342F5FF3FE105310521051B
:105F400011F1E8940894E795D901AA2329F4AB2F1D
:105F5000BE2FF85FD0F310C0FF5F70F4A695E0F796
:105F6000F73950F019F0FF3A38F49F779F930CD02F
:105F70000F9007FC905808953EF014CF60E070E059
:105F800080E89FE308954FE79F775F934F933F9398
:105F90002F93A2D02F913F914F915F9152DF09C073
:105FA000D7DE880B990B089519F40EF0F5CE3ECF8D
:105FB000F9CE22DFC8F39638C0F707F80F92E894BD
:105FC0002BE33AEA48EB5FE74ADF0F920F920F921A
:105FD0004DB75EB70F92C0D0E0EEF0E016D04F9113
:105FE0005F91EF91FF91E595EE1FFF1F49F0FE577E
:105FF000E0684427EE0F441FFA95E1F74195550BF1
:1060000032D00F9007FE26C00895DF93CF931F93E1
:106010000F93FF92EF92DF927B018C01689405C091
:10602000DA2EEF011ADFFE01E894A5912591359152
:1060300045915591AEF3EF015EDDFE019701A80198
:10604000DA9479F7DF90EF90FF900F911F91CF9145
:10605000DF9108959B01AC0160E070E080E89FE370
:10606000A1CD9ACEACC0C8DEE8F39923D9F3940F42
:10607000511DBBF39150504094F059F0882332F0F9
:10608000660F771F881F91505040C1F79E3F510502
:1060900044F7880F911D9695879597F908955F3F6E
:1060A000ACF0983E9CF0BB27869577956795B795A1
:1060B00008F4B1609395C1F7BB0F58F711F460FF76
:1060C000E8CF6F5F7F4F8F4F9F4FE3CFB0CE0EF083
:1060D00076C068CE689460CE8FDEC8F39923D1F382
:1060E000C6F3DF93CF931F930F93FF92C92FDD2742
:1060F00088232AF02197660F771F881FDAF720E0A0
:1061000030E040E85FEB9FE3883920F0803E30F0DC
:1061100021968F77DFDCE8E0F1E003C0DBDCE5E32C
:10612000F1E073DF8B01BE01EC01FB2E6F577109AB
:106130007595771F880B990BD0DD28E132E741E395
:106140005FE38BDEAF2D9801AE01FF900F911F91A1
:10615000CF91DF91D0DC37CEFA01DC01AA0FBB1F53
:106160009B01AC01BF5728F42227332744275078DE
:106170001FC0B75188F4AB2F00244695379527955B
:10618000011CA395D2F3002069F0220F331F441F96
:10619000B395DAF30DD09DCC61307105A0E88A0784
:1061A000B94630F49B01AC016627772788279078A1
:1061B000309621F0208331834283538308959F3F9B
:1061C00031F0915020F4879577956795B795880FB2
:1061D000911D9695879597F90895DB018F939F936D
:1061E0000E944431BF91AF91A29F800D911DA39F4A
:1061F000900DB29F900D11240895A1E21A2EAA1BB2
:10620000BB1BFD010DC0AA1FBB1FEE1FFF1FA21766
:10621000B307E407F50720F0A21BB30BE40BF50B63
:10622000661F771F881F991F1A9469F760957095EC
:10623000809590959B01AC01BD01CF010895052E7D
:1062400097FB1EF400940E94363157FD07D00E9440
:10625000FD3007FC03D04EF40C9436315095409538
:10626000309521953F4F4F4F5F4F08959095809502
:10627000709561957F4F8F4F9F4F0895EE0FFF1FD1
:106280000590F491E02D09940E945731A59F900D3F
:10629000B49F900DA49F800D911D11240895B7FF08
:1062A0000C9444310E944431821B930B0895A29FA9
:1062B000B001B39FC001A39F700D811D1124911DDA
:1062C000B29F700D811D1124911D0895CF93DF930E
:1062D0008230910510F482E090E0E0918F06F09119
:1062E000900620E030E0A0E0B0E0309739F1408146
:1062F000518148175907B8F04817590771F482813E
:106300009381109729F013969C938E9312972CC02B
:106310009093900680938F0627C02115310531F0A8
:106320004217530718F0A901DB0101C0EF019A01E0
:10633000BD01DF010280F381E02DD7CF21153105AA
:10634000F9F0281B390B2430310580F48A819B81B8
:106350006115710521F0FB019383828304C0909342
:10636000900680938F06FE01329644C0FE01E20F34
:10637000F31F8193919322503109398328833AC0C6
:1063800020918D0630918E06232B41F4209102013D
:106390003091030130938E0620938D0620910001E9
:1063A000309101012115310541F42DB73EB74091DF
:1063B000040150910501241B350BE0918D06F091ED
:1063C0008E06E217F307A0F42E1B3F0B28173907A0
:1063D00078F0AC014E5F5F4F2417350748F04E0F41
:1063E0005F1F50938E0640938D068193919302C058
:1063F000E0E0F0E0CF01DF91CF910895CF93DF93FC
:10640000009709F487C0FC01329713821282C09171
:106410008F06D0919006209781F420813181280F3A
:10642000391F80918D0690918E068217930779F51A
:10643000F0938E06E0938D066DC0DE0120E030E023
:10644000AE17BF0750F412964D915C9113979D01C2
:106450004115510509F1DA01F3CFB383A2834081DD
:106460005181840F951F8A179B0771F48D919C9120
:106470001197840F951F02969183808312968D91B8
:106480009C911397938382832115310529F4F0930E
:106490009006E0938F063EC0D9011396FC93EE93CD
:1064A00012974D915D91A40FB51FEA17FB0779F480
:1064B00080819181840F951F0296D90111969C933A
:1064C0008E938281938113969C938E931297E0E032
:1064D000F0E08A819B81009719F0FE01EC01F9CF71
:1064E000CE01029628813981820F931F20918D065B
:1064F00030918E062817390769F4309729F41092E5
:10650000900610928F0602C013821282D0938E06DC
:10651000C0938D06DF91CF910895A0E0B0E0E3E94C
:10652000F2E30C944536EC01CB01209719F40E945C
:106530006631B8C0FE01E60FF71F9E0122503109F7
:10654000E217F30708F4ACC0D9010D911C91119723
:1065500006171707B8F00530110508F49FC0A80109
:10656000445051094617570708F498C002501109C2
:10657000061B170B019311936D937C93CF010E941F
:10658000FE318CC05B01A01AB10A4E01800E911E33
:10659000A0918F06B0919006612C712C60E070E0A4
:1065A000109709F449C0A815B905C9F5ED90FC90FC
:1065B0001197670142E0C40ED11CCA14DB0478F1C4
:1065C00047018A189B08640142E0C40ED11C129650
:1065D000BC9012971396AC91B5E0CB16D10440F065
:1065E000B282A38391828082D9018D939C9309C04A
:1065F0000E5F1F4F0E0D1F1DF90111830083EB2D40
:10660000FA2F6115710531F0DB011396FC93EE93BF
:10661000129744C0F0939006E0938F063FC06D91AF
:106620007C9111976616770608F43B01BD0112961E
:106630000D90BC91A02DB4CF60918D0670918E0607
:1066400068157905E9F468167906D0F440910001DF
:10665000509101014115510541F44DB75EB760916C
:10666000040170910501461B570BE417F507C0F4B0
:10667000F0938E06E0938D06F901918380830EC01E
:106680000E9466317C01009759F0A801BE010E946A
:106690005733CE010E94FE31C70104C0CE0102C0B3
:1066A00080E090E0CDB7DEB7EEE00C946136FB0100
:1066B000DC0102C001900D9241505040D8F708957E
:1066C000FB01DC0101900D920020E1F708954532B5
:1066D000510520F4423010F00C947233FB0110820B
:1066E000CB010895BB274A3031F4992322F4BDE24F
:1066F000909581959F4F0C947E33BB27FB015527C6
:10670000AA27880F991FAA1FA41710F0A41B83950E
:106710005051B9F7A05DAA3308F0A95DA193009785
:1067200079F7B111B1931192CB010C94A135AEE080
:10673000B0E0EDE9F3E30C944F360D891E8986E055
:106740008C831A8309838FEF9FE79E838D83AE012D
:10675000475E5F4F6F89788DCE0101960E94B933F5
:10676000EF81F885E00FF11F10822E96E4E00C9483
:106770006B36ACE0B0E0EFEBF3E30C9441367C0118
:106780006B018A01FC0117821682838181FFBDC1E2
:10679000CE0101964C01F7019381F60193FD85919D
:1067A00093FF81916F01882309F4ABC1853239F4DD
:1067B00093FD859193FF81916F01853229F4B70193
:1067C00090E00E94B135E7CF512C312C20E02032EF
:1067D000A0F48B3269F030F4803259F0833269F4DE
:1067E00020612CC08D3239F0803339F4216026C00D
:1067F0002260246023C0286021C027FD27C030ED1F
:10680000380F3A3078F426FF06C0FAE05F9E300D6C
:106810001124532E13C08AE0389E300D1124332EDC
:1068200020620CC08E3221F426FD6BC1206406C0AC
:106830008C3611F4206802C0883641F4F60193FDCD
:10684000859193FF81916F018111C1CF982F9F7D19
:106850009554933028F40C5F1F4FFFE3F9830DC06C
:10686000833631F0833771F0833509F05BC022C085
:10687000F801808189830E5F1F4F44244394512C7B
:10688000540115C03801F2E06F0E711CF801A080B0
:10689000B18026FF03C0652D70E002C06FEF7FEF6F
:1068A000C5012C870E9496352C0183012C852F77FA
:1068B000222E17C03801F2E06F0E711CF801A08083
:1068C000B18026FF03C0652D70E002C06FEF7FEF3F
:1068D000C5012C870E948B352C012C852068222E27
:1068E000830123FC1BC0832D90E048165906B0F4A9
:1068F000B70180E290E00E94B1353A94F4CFF501FF
:1069000027FC859127FE81915F01B70190E00E94ED
:10691000B13531103A94F1E04F1A51084114510445
:1069200071F7E5C0843611F0893639F5F80127FF93
:1069300007C060817181828193810C5F1F4F08C005
:1069400060817181882777FD8095982F0E5F1F4F9A
:106950002F76B22E97FF09C090958095709561951E
:106960007F4F8F4F9F4F2068B22E2AE030E0A40166
:106970000E94E335A82EA81844C0853729F42F7E3D
:10698000B22E2AE030E025C0F22FF97FBF2E8F36DD
:10699000C1F018F4883579F0B4C0803719F0883721
:1069A00021F0AFC02F2F2061B22EB4FE0DC08B2D71
:1069B0008460B82E09C024FF0AC09F2F9660B92EAC
:1069C00006C028E030E005C020E130E002C020E150
:1069D00032E0F801B7FE07C0608171818281938146
:1069E0000C5F1F4F06C06081718180E090E00E5FF8
:1069F0001F4FA4010E94E335A82EA818FB2DFF7796
:106A0000BF2EB6FE0BC02B2D2E7FA51450F4B4FE66
:106A10000AC0B2FC08C02B2D2E7E05C07A2C2B2D6F
:106A200003C07A2C01C0752C24FF0DC0FE01EA0DB5
:106A3000F11D8081803311F4297E09C022FF06C038
:106A40007394739404C0822F867809F0739423FDA5
:106A500013C020FF06C05A2C731418F4530C571897
:106A6000732C731468F4B70180E290E02C870E94C5
:106A7000B13573942C85F5CF731410F4371801C019
:106A8000312C24FF12C0B70180E390E02C870E94D4
:106A9000B1352C8522FF17C021FF03C088E590E0A7
:106AA00002C088E790E0B7010CC0822F867859F0C9
:106AB00021FD02C080E201C08BE227FD8DE2B7011B
:106AC00090E00E94B135A51438F4B70180E390E05E
:106AD0000E94B1355A94F7CFAA94F401EA0DF11D42
:106AE0008081B70190E00E94B135A110F5CF33202D
:106AF00009F451CEB70180E290E00E94B1353A949A
:106B0000F6CFF7018681978102C08FEF9FEF2C9619
:106B1000E2E10C945D36FC0105906150704001107B
:106B2000D8F7809590958E0F9F1F0895FC016150B6
:106B3000704001900110D8F7809590958E0F9F1F9F
:106B40000895DC01FC01672F71917723E1F73297FB
:106B500004C07C916D9370836291AE17BF07C8F338
:106B600008950F931F93CF93DF93182F092FEB01F5
:106B70008B8181FD03C08FEF9FEF20C082FF10C08B
:106B80004E815F812C813D81421753077CF4E8815F
:106B9000F9819F012F5F3F4F39832883108306C0FF
:106BA000E885F985812F0995892B29F72E813F8169
:106BB0002F5F3F4F3F832E83812F902FDF91CF9107
:106BC0001F910F910895FA01AA27283051F1203121
:106BD00081F1E8946F936E7F6E5F7F4F8F4F9F4F71
:106BE000AF4FB1E03ED0B4E03CD0670F781F891FB3
:106BF0009A1FA11D680F791F8A1F911DA11D6A0F81
:106C0000711D811D911DA11D20D009F468943F9133
:106C10002AE0269F11243019305D3193DEF6CF0132
:106C20000895462F4770405D4193B3E00FD0C9F7F8
:106C3000F6CF462F4F70405D4A3318F0495D31FD65
:106C40004052419302D0A9F7EACFB4E0A6959795B8
:106C5000879577956795BA95C9F70097610571058E
:106C600008959B01AC010A2E0694579547953795D8
:106C70002795BA95C9F7620F731F841F951FA01D32
:106C800008952F923F924F925F926F927F928F92D0
:106C90009F92AF92BF92CF92DF92EF92FF920F93AB
:106CA0001F93CF93DF93CDB7DEB7CA1BDB0B0FB6B5
:106CB000F894DEBF0FBECDBF09942A883988488872
:106CC0005F846E847D848C849B84AA84B984C88408
:106CD000DF80EE80FD800C811B81AA81B981CE0FFF
:106CE000D11D0FB6F894DEBF0FBECDBFED010895E4
:046CF000F894FFCF46
:106CF4000000910680006B25000059430000030347
:106D0400CC3F0D00594300000A5B004C6143726F95
:106D14007373654954506C75735265616465720090
:106D240031302E31710020663A0020743A007E0022
:106D340020723A002900202B202800202B20424DCD
:106D440050313830000A456E642072656365697697
:106D5400696E672C204845582072617720646174FD
:106D6400613A200052656C61796564002A2A2A2000
:106D74004C6143726F7373652077656174686572E3
:106D84002073746174696F6E20776972656C6573C2
:106D94007320726563656976657220666F72204937
:106DA400542B2073656E736F7273202A2A2A005243
:106DB4006164696F20736574757020636F6D706CA6
:106DC4006574652E205374617274696E6720746FE4
:106DD4002072656365697665206D657373616765A7
:106DE40073004F4B2043432000437573746F6D53FE
:106DF400656E736F72205B005D2000204352433A3E
:106E040057524F4E4700204352433A4F4B002049BC
:106E1400443A307800204E62724F66446174614295
:106E2400797465733A0020446174613A00204352D6
:106E3400433A307800253036642000454D543731CC
:106E44003130205B005D0020533A002049443A0071
:106E540020563A00206D413A0020573A00206B57E3
:106E6400683A0020436F6E2E3A0020506169723AEE
:106E740000204352433A004F4B20454D54373131A3
:106E84003020004F4B205753200020320020323551
:106E94003520323535004F4B20392000204E6577A0
:106EA400426174743A002042697431323A002054C9
:106EB400656D703A00205765616B426174743A00E5
:106EC4002048756D3A004C6143726F737365205BA3
:106ED40000232320435243204641494C20232300CE
:106EE4004E6F2076616C6964207374617274004E15
:106EF4006F2076616C69642054656D70657261748D
:106F04007572653A20004E6F2076616C6964204C7E
:106F14006576656C3A20004E6F2076616C6964205A
:106F2400566F6C746167653A20004C6576656C53E6
:106F3400656E646572205B00204C6576656C3A0072
:106F440020566F6C743A004F4B204C532000203075
:106F5400200073706931363A00577269746552655E
:106F6400673A002D3E0052464D31320052464D36AE
:106F740039004E6F6E6500526164696F2069733A1F
:106F8400200053656E64696E6720646174613A2001
:106F940000545833384954205B00000000000F1D92
:106FA400E21CB71CBF1CD21CE11C54583232495499
:106FB4000057533130383000204C6F77426174747D
:106FC4003A00204572726F723A002D2D2D00205226
:106FD40061696E3A002057696E643A002066726FE8
:106FE4006D3A0020477573743A00206D2F730000CA
:106FF4000000003028AC29B227CB27BD270E286E0D
:0E700400616E00696E66006F7666002E0000F9
:00000001FF
